:020000041001E9
:1080000000D0003043AC0110D9AB0110D9AB011046
:108010000000000000000000000000000000000060
:10802000000000000000000000000000D9AB0110BB
:108030000000000000000000D9AB0110D9AB011016
:10804000D9AB0110D9AB0110D9AB0110D9AB0110DC
:10805000D9AB0110D9AB0110D9AB0110D9AB0110CC
:10806000D9AB0110D9AB0110D9AB0110D9AB0110BC
:10807000D9AB0110D9AB0110D9AB0110D9AB0110AC
:10808000D9AB0110D9AB0110D9AB0110D9AB01109C
:10809000D9AB0110D9AB0110D9AB0110D9AB01108C
:1080A000D9AB0110D9AB0110D9AB0110D9AB01107C
:1080B000D9AB0110D9AB0110D9AB0110D9AB01106C
:1080C000D9AB0110D9AB0110D9AB0110D9AB01105C
:1080D000D9AB0110D9AB0110D9AB0110D9AB01104C
:1080E000D9AB0110D9AB0110D9AB0110D9AB01103C
:1080F000D9AB0110D9AB0110D9AB0110D9AB01102C
:10810000D9AB0110D9AB0110D9AB0110D9AB01101B
:10811000D9AB0110D9AB0110D9AB0110D9AB01100B
:10812000D9AB0110D9AB0110D9AB0110D9AB0110FB
:10813000D9AB0110D9AB0110D9AB0110D9AB0110EB
:10814000D9AB0110D9AB0110D9AB0110D9AB0110DB
:10815000D9AB0110D9AB0110D9AB0110D9AB0110CB
:10816000D9AB0110D9AB0110D9AB0110D9AB0110BB
:10817000D9AB0110D9AB0110D9AB0110D9AB0110AB
:10818000D9AB0110D9AB0110D9AB0110D9AB01109B
:10819000D9AB0110D9AB0110D9AB0110D9AB01108B
:1081A000D9AB0110D9AB0110D9AB0110D9AB01107B
:1081B000D9AB0110D9AB0110D9AB0110D9AB01106B
:1081C000D9AB0110D9AB0110D9AB011057AC0110DC
:1081D000D9AB0110D9AB0110D9AB0110D9AB01104B
:1081E000D9AB0110D9AB0110D9AB0110D9AB01103B
:1081F000D9AB0110D9AB0110D9AB0110D9AB01102B
:10820000D9AB0110D9AB0110D9AB0110D9AB01101A
:1082100000F002F800F0B5F80CA030C808382418B7
:108220002D18671EA246AB4654465D46AC4201D1AE
:1082300000F0A7F87E460F3EB6460FCC012633422B
:1082400000D0FB1A3343A246AB461847908A000081
:10825000B08A00000023002400250026103A01D334
:1082600078C1FBD8520700D330C100D50B607047EE
:1082700010B56E2902D100F08CFE10BD702902D11C
:1082800000F0A9FA10BD662902D107F0E3FA10BD8B
:10829000652902D107F0DEFA10BD672902D107F087
:1082A000D9FA10BD612902D107F0DCFA10BD0368CC
:1082B0001B0A01D380231943692902D100F016FA61
:1082C00010BD642902D100F011FA10BD752902D148
:1082D00000F00CFA10BD6F2902D100F075FF10BD3F
:1082E000782902D100F064FA10BDE92902D100F02A
:1082F00011FF10BDE42902D100F00CFF10BDF529DB
:1083000002D100F007FF10BDEF2902D100F068FF95
:1083100010BDF82902D100F059FA10BD0368DB093D
:1083200001D380231943632902D100F075FE10BDEB
:10833000732902D100F078FE10BDE32902D101F0CB
:1083400056FE10BDF32902D101F059FE10BD0020E8
:1083500010BD1FB50098019900F07DFD01F080FE71
:1083600004000020002107F049FA401C6060002052
:10837000002107F059FAE06001F0F8F800F03AFD4A
:108380001FBD0648854603B405F026F903BC02F07C
:1083900069FA02F07BFA05F044FC000000D00030DE
:1083A00070B505460C46164602E00FCC0FC5103ED0
:1083B000102EFAD2082E02D303CC03C5083E042E99
:1083C00007D301CC01C5361F03E021782970641C56
:1083D0006D1C761EF9D270BD7047000000487047D2
:1083E00044D3003070B5064600F018FD05683046ED
:1083F0000B30C408E400B44201D8002070BD6868A6
:108400002A46002818D00168A14211D30B46214604
:1084100008318B4208D3436801194B6003681B1B6A
:108420000B605160046001E041685160001D70BD47
:10843000024640680028E6D12146284600F0F6FCB6
:108440000028DCD170BD70B50446051F00F0E6FCC5
:108450000068002C1AD0446801E020466468002CB3
:1084600001D0AC42F9D301680A18AA4204D12A68A3
:1084700005468918016000E0456028684119A1425D
:1084800005D16168696021684018286070BD6C6022
:1084900070BD10B5202A04DB0146203A914000202F
:1084A00010BD914020239C1A0346E340194390409D
:1084B00010BD10B5202A04DB0846203AD040002128
:1084C00010BD0B462024D340D040A21A914008434F
:1084D000194610BD4343514330B55C18010C130CD1
:1084E0000D4692B25D4380B251432C190546554367
:1084F0000A0C09044D1962415843010C000440194B
:10850000514130BDFEB5054610460C46184373D0A8
:10851000AE468C460020AD1A01469C4167D36646A4
:10852000002701243D46B61A9D4102D313463A4620
:108530002124654676462F04360C3E432D0CB61A90
:108540009D4104D3150C1B042B43120410346546C3
:1085500076462F06360A3E432D0AB61A9D4104D3AD
:10856000150E1B022B4312020834654676462F0770
:1085700036093E432D09B61A9D4104D3150F1B0140
:108580002B431201241D65467646AF07B6083E43CD
:10859000AD08B61A9D4104D3950F9B002B43920062
:1085A000A41C65467646EF0776083E436D08B61A6A
:1085B0009D411AD392185B41641C16E00018764660
:1085C00065464941B71A9D410191009009D3604623
:1085D000B11A98418E468446009801990025401CA6
:1085E0006941DD0752082A435B08641EE6D57246DE
:1085F000634603B0F0BDFFE700200146C046C04619
:108600002A462346F5E710B50B460146184600F00A
:108610000FFD10BD7CB51D4616460C00009001D024
:108620000019401E084B7B442A466946019030469B
:1086300000F0C7FC002C054603D06946002000F07E
:10864000D3FC28467CBD0000C909000070B5044673
:1086500085690068C10601D5302600E02026C007E4
:1086600007D070BD62683046A1689047206A401C00
:1086700020626D1EF6D570BD70B504468569007820
:10868000C00707D170BD6268A16820209047206AAA
:10869000401C20626D1EF6D570BD70B50C460546B7
:1086A000012A05D02878800600D5EA69002302E077
:1086B000012305E05B1C934202D2E05C0028F9D163
:1086C000A869E618C01AA861286AC0182862284656
:1086D000FFF7BCFF04E06A682078A968641C904733
:1086E000B442F8D32846FFF7C7FF70BDF7B50025A1
:1086F00075291068009914A611D000F0E0FB00283D
:1087000002DA404211A608E0009909688A0701D5FB
:108710000FA602E0490704D50EA6012501E000F0EE
:10872000D7FB009F0024243704E001F06AF83031C1
:108730003955641C0028F8D12B4632462146009852
:1087400000F0CFFBFEBD0000000000002D00000087
:108750002B00000020000000F8B50F460188090535
:1087600002D5224C7C4402E0204C7C440E34054669
:108770000021243508E016071209360FA65D6E5455
:108780001E0732431B09491C16461E43F3D12246DD
:1087900004780023240705D5702F06D0002901D0C6
:1087A0000223113200F09DFBF8BD01231032F9E7DE
:1087B00070B504460D462146106800F089FB002381
:1087C000024629462046FFF7C7FF70BDD21DD308D9
:1087D000DB000CCBC0E730B40368202412682343CD
:1087E00003600823C36130BC0023B5E70C710000AF
:1087F000F3B50446002081B020622046E168884736
:10880000002872D0252802D06268A168ABE0594FD9
:1088100000267F442046E16888472028054608DB7B
:10882000312D06D2781920380078002801D006436F
:10883000F0E7B00701D5042086430020E061074639
:10884000A0612A2D0AD0284606F0C2FF002827D0B2
:10885000B8000019303D0090856119E00298BA0017
:10886000121902C8916102902046E1688847012FE1
:10887000054617D1E06900281FDA202086431CE056
:1088800000980A218069484300994019303888616E
:108890002046E1688847054606F09AFF0028EFD198
:1088A000012F0AD02E2D08D12046E16888470546C1
:1088B000202006437F1C022FC3DBA069002803DAB7
:1088C0004042A06101200643F00701D010208643FA
:1088D0006C2D0BD0682D09D04C2D3CD06A2D38D092
:1088E000742D38D07A2D36D016E040E0E1682F465E
:1088F00020468847B842054609D16C2F29D001206F
:108900008002E168064320468847054604E06C2F54
:108910001DD0FF2001300643002D28D028464138C5
:10892000192803D80120C0020643203520462660BE
:108930002946029A1646FFF79BFC002810D0012812
:108940000BD0F61DF008C0000830029055E740201B
:10895000E1E78020D5E70020D3E7361D02964CE7FB
:1089600062682846A1689047206A401C44E7206A54
:10897000FEBD000086700000F8B5044616460D46A0
:108980004769007B800730D0384604F04DFE002850
:108990002BD132461026002A25D0012A02D0022AE5
:1089A00023D104E0204600F021FD45191BE03846A4
:1089B00004F027FEE16831430028E16004DA204634
:1089C00000F05CFD0120F8BDC9030BD56268E16AC7
:1089D000914200D81146A26989182269891A8142F8
:1089E00000DD08462D18002D01DA0220F8BDE16AED
:1089F0006068E268814206D29103E06203D50121FA
:108A000049048A433243A669AE4211DCE16A8142DD
:108A100001D90B4600E003469F192369FF1AAF42B4
:108A200006DD814201D90F4600E007469F4206D18C
:108A3000202002430020A060A56220600DE0AD1B55
:108A4000E669AE1B8142A66000D90846C01A281A02
:108A500020605819606020208243034802400020B3
:108A6000E26040342072F8BDBFCFD7FFF7B516469D
:108A70000C46104600F06EF82078611C61280AD080
:108A8000722802D0772839D102E00125002404E0C1
:108A90000225042401E02D4D08240222032301278E
:108AA0000878491C2B2806D0622807D02039C87FB7
:108AB000742807D008E01D431443F1E70420054360
:108AC0003C43EDE7102004430098214604F0AEFD3E
:108AD000411C13D00021316171600121F560490210
:108AE000F1617061200704D5304602220021FFF7B2
:108AF00043FF306D384330653046FEBD0020FEBD7B
:108B0000F8B50D460646124C206DC10704D0410849
:108B100004D044086400F7E7224610E05420FFF731
:108B200061FC070010D07908206D49000122114333
:108B3000084354212065384600F011F93A46294689
:108B40003046FFF793FFF8BD0020F8BD028000001B
:108B500048D30030FEB50446466900690F4F0190C6
:108B6000E56800200090A80707D0204600F0B6FC7A
:108B7000304604F043FD002801DA3846FEBD2805E2
:108B800002D50198FFF75FFC4C21204600F0E7F882
:108B9000206D4008400020650098FEBDFFFFFFFFEC
:108BA00030B503461D78002D08D00A461478521CB3
:108BB000002C03D0AC42F9D15B1CF3E7181A30BD8E
:108BC000034610B50B439B070FD1042A0DD308C8E9
:108BD00010C9121FA342F8D018BA21BA884201D98D
:108BE000012010BD0020C04310BD002A03D0D307D0
:108BF00003D0521C07E0002010BD03780C78401C05
:108C0000491C1B1B07D103780C78401C491C1B1BFB
:108C100001D1921EF1D1184610BD000030B5441CA0
:108C200003E00178401C00290DD08107F9D10B4BDE
:108C3000DD0104C8D11A91432940FAD0001B0A066D
:108C400003D0C01E30BD001B30BD0A0401D0801E01
:108C500030BD0902FCD0401E30BD00000101010101
:108C6000F8B5042A2CD3830712D00B78491C037063
:108C7000401C521E83070BD00B78491C0370401C0C
:108C8000521E830704D00B78491C0370401C521EEF
:108C90008B079B0F05D0C91ADF002023DE1B08C9F4
:108CA0000AE0FFF77DFBF8BD1D4608C9FD401C46E4
:108CB000B4402C4310C0121F042AF5D2F308C91A7D
:108CC000521EF0D40B78491C0370401C521EEAD48B
:108CD0000B78491C0370401C012AE4D40978017008
:108CE000F8BD134610B50446CAB2194610028218E0
:108CF00010048218204600F021F8204610BDD2B2A0
:108D000010B513029A1813049A1800F017F810BD42
:108D1000D2B210B513029A1813049A1800F001F891
:108D200010BD01E004C0091F0429FBD28B0701D547
:108D30000280801CC90700D00270704700290BD048
:108D4000C30702D00270401C491E022904D38307C6
:108D500002D50280801C891EE3E70022EEE7002294
:108D6000DFE70000024670B50A4392072AD11E4D84
:108D7000EE0104C808C9541B9443344017D0D0B244
:108D8000D9B2401A2106014310D190B299B2401ACB
:108D9000210401430AD110021902000A090A401AEB
:108DA0002102014302D1100E190E401A70BD9A42E1
:108DB000DFD010BA19BA884201D9012070BD002055
:108DC000C04370BD02780B78401C491C002A09D0B2
:108DD0009A4207D102780B78401C491C002A01D026
:108DE0009A42EFD0D01A70BD01010101704770475F
:108DF0007047000070B5064C7C44064D7D4403E08E
:108E0000206800198047241DAC42F9D170BD0000D4
:108E10002C8000002C800000704700000048704744
:108E200044D40030704770477047704738B50446E7
:108E30000A4600206946C046C046002805D00246C2
:108E40002046009900F0FAFC012038BD10B5012041
:108E500001F000F910BDF8B5C046C0460546002037
:108E60000C461020C0460646A819A0420DD932462D
:108E700069460020C046C046070001D101F0EAF86B
:108E80000098A04200D00546C419FFF7C7FFF61DA1
:108E900007460560F008C0004619284600F008F8AB
:108EA000B44204D031463868A21B00F0C7FCF8BDBC
:108EB00000210160416080607047102070470968A0
:108EC0004A0501D540B27047C905FCD500B27047CC
:108ED00009684A0501D5C0B27047C905FCD580B202
:108EE0007047FFB504460D4681B0243000902168DC
:108EF000880604D51022E0699143216000E001203A
:108F0000A84201DD471B00E000270498A1697A19F7
:108F10001018081AA0612078C00602D42046FFF776
:108F200095FB002608E003986268A168805D904781
:108F3000206A401C761C206204988642F3DB20786D
:108F4000C0060AD52046FFF781FB06E06268A168EB
:108F500030209047206A401C206238467F1E00283F
:108F6000F4DC07E000986268A168405D9047206AE1
:108F7000401C206228466D1E0028F3DC2046FFF7C7
:108F80007BFB2078000602D5022005B0F0BD012051
:108F9000FBE711680268006A530501D5087009E013
:108FA000D30501D5088005E0130602D5C21705C117
:108FB00000E008600120704701694A1C02610878DE
:108FC000704700B58FB002910021059105490193CA
:108FD00079440391114604906846FFF709FC0FB0ED
:108FE00000BD0000E5FFFFFF0A681070521C0A6018
:108FF00070470CC908399A4202D2531C0B6010709A
:10900000704710B54369002B02D0C046C04601E04E
:10901000FFF743FB012010BD1278014624310A708E
:1090200000224A700122ECE711680022D243E8E7EF
:10903000084B70B50D467B44FFF7C3FF0446284636
:1090400000F0D8F8002802D00020C04370BD2046B0
:1090500070BD0000A5670000F7B50446154686B050
:109060002B487844002703C83E460090019111E048
:1090700007986A467100415A02A800F0C4FF411CDB
:1090800007D02178890603D5E269391891420ED8B4
:109090003F18761C2078800602D5E069B84206DDCC
:1090A000AE42E5DB07987100405A0028E0D1A06984
:1090B000C01BA0612046FFF7C9FA154878445A380A
:1090C00003C800900020019116E041006A4607980D
:1090D000415A02A800F097FF0590401C0AD00025D5
:1090E00005E0626802A8A168405D90476D1C059884
:1090F0008542F6D30498401CB0420490E5DB206A18
:10910000C01920622046FFF7B7FA09B0F0BD000091
:109110004A680000F7B5D21D0025D20815A6D20076
:10912000F52905CA11D0002A05DA002140429141F3
:1091300011A60A4608E0009909688B0701D50FA619
:1091400002E0490701D50EA601251146009F002423
:10915000243704E000F08CFB30323A55641C0246A0
:109160000A43F7D12B46324621460098FFF7B9FE55
:10917000FEBD0000000000002D0000002B000000DC
:109180002000000070B504460021243408E0550793
:10919000D2086D0F303565545D072A43DB08491C42
:1091A00015461D43F3D10468002310A2250708D5F6
:1091B00020252C400C4304D0C46901230CA2641E5A
:1091C000C461FFF78EFE70BD10B5044621461068DD
:1091D000FFF77EFE002302462046FFF7D3FF10BDB7
:1091E000D21DD108C9000CC9CCE700000000000066
:1091F00030000000C068802108407047F8B505467F
:109200000C46C8680521C904884301218905084323
:10921000E060800602D5204600F086F97149E068DA
:109220000140022903D0204600F028F9BCE00521C6
:10923000012249030140D20391420FD1C00306D558
:109240006168E06A884200D80846606006E02069EC
:10925000E0626060606904F0D4F9A061A168002256
:10926000EEB200290EDAE06883050BD4C943A16091
:109270000921226049030843E0606068411C616085
:109280000670ACE0E068012149030843E06000207B
:1092900020602069002831D1606904F0C5F90125FA
:1092A00027462437ED02002816D0A0898005800FBC
:1092B00008D0E069FFF796F80028206102D0E06846
:1092C000284318E001202761E061E06803210902DA
:1092D0008843012189020DE0E069FFF783F8002847
:1092E0002061EFD0E0682843E0608105890F03D159
:1092F000FF2101310843E06020696060E2683A4F75
:109300002569D0051FD56168E06A884200D8084603
:10931000411B05D02246284600F0BAF8002843D168
:10932000E068010204D5E56200206560A06053E0BA
:10933000691CE1626160E169491E3843A160E06037
:1093400030462E70F8BD100201D53A4009E0606841
:10935000411C61600670E06838430A2EE06006D068
:109360000022E16A6068814203D90B4602E00122D3
:10937000F7E70346A7895B1B7F0504D4E7699F4293
:1093800001DD002A1ED0814200D801460F1A0020BC
:10939000E5626560002BA06009DD2246194628467B
:1093A00000F076F8002802D00020C043F8BD002F5E
:1093B00008D0A069E5626560C01BA061E06810216B
:1093C0000843E060E068000209D56168A069E562D1
:1093D000491B40186560A0610120C043F8BD3046BC
:1093E000F8BD0000821000000000010010B5014629
:1093F000C268900703D0900607D5886A0AE0FEF796
:10940000EDFF01210160881E10BD8B694868C018FE
:109410000B69C01A40310B7A002B02D0497A401AEE
:1094200010BD1103FCD50028FADD401E10BD000060
:1094300070B5C468A50713D0650211D4D51FF93DD6
:109440000AD0FF3D6D1E07D0FF3DFF3D022D07D125
:1094500001462431012305E0074E5D1EB54201D3CC
:10946000012070BD0161C36141600F2109028C437D
:109470001443C460002070BDFFFFFF00C16880225C
:10948000114392039143C1600021816001607047E4
:10949000F7B514460E463348D5685769054209D0DA
:1094A0003846A16904F00EF9002811DB2D48C043AD
:1094B0000540E5602B4632463846009904F005F930
:1094C0004200A1695208B21A89180028A16104D08B
:1094D0002046FFF7D3FF0020C043FEBD70B5044611
:1094E0000569C06A6168884200D80846E1680522BB
:1094F000D2049143E160C90314D5A84209D02246A1
:10950000411B2846FFF7C4FF002802D00020C043BB
:1095100070BDE56200206560A060E068012109047B
:109520008843E060002070BD10B50446C06820216B
:109530008843E060A16AA06988420ED02046FFF708
:10954000CDFFE06803210903884310210843E06050
:10955000A06AA0612069E06260600349E068084099
:10956000E06010BD10000200BFBFFFFF10B5434810
:109570005421FFF7F4FB42485421FFF7F0FB414828
:109580005421FFF7ECFB40483C493D4B404A016009
:109590003E4803603B4810605A1C0A65411C19652F
:1095A000012101653C48354A3AA17844FFF75EFA4B
:1095B000002804D1384878440C3800F045FD38487C
:1095C0002F4A36A17844FFF751FA002804D13448D5
:1095D00078440C3800F038FD32482A4A2FA17844EC
:1095E000FFF744FA002804D12E4878440C3800F0E4
:1095F0002BFD40232148DC0000212246FFF718FF05
:10960000002804D0244878445C3800F01DFD1C4834
:10961000224640230021FFF70BFF002804D02048FA
:1096200078445C3800F010FD1648224610230021D3
:10963000FFF7FEFE002804D01A4878445C3800F09A
:1096400003FD10BD0F4870B5006D44080B48640061
:10965000FFF780FA0A48FFF77DFA0A48FFF77AFA1F
:1096600009E0206D450820466D00FFF773FA20469B
:10967000FEF7E9FE2C46002CF3D170BD48D3003034
:109680009CD30030F0D3003010D2003014D2003020
:1096900018D2003072000000267000007700000031
:1096A00013700000EA6F0000002203098B422CD3E4
:1096B000030A8B4211D300239C464EE003460B4322
:1096C0003CD4002243088B4231D303098B421CD384
:1096D000030A8B4201D394463FE0C3098B4201D376
:1096E000CB01C01A524183098B4201D38B01C01AAE
:1096F000524143098B4201D34B01C01A5241030925
:109700008B4201D30B01C01A5241C3088B4201D3D3
:10971000CB00C01A524183088B4201D38B00C01A80
:10972000524143088B4201D34B00C01A5241411AA7
:1097300000D201465241104670475DE0CA0F00D08A
:109740004942031000D3404253409C460022030983
:109750008B422DD3030A8B4212D38901FC2212BA09
:10976000030A8B420CD3890192118B4208D38901E1
:1097700092118B4204D389013AD0921100E08909F9
:10978000C3098B4201D3CB01C01A524183098B42DA
:1097900001D38B01C01A524143098B4201D34B01C3
:1097A000C01A524103098B4201D30B01C01A524126
:1097B000C3088B4201D3CB00C01A524183088B42AD
:1097C00001D38B00C01A5241D9D243088B4201D336
:1097D0004B00C01A5241411A00D201465241104674
:1097E00063465B1001D34042002B00D549427047CD
:1097F00063465B1000D3404201B50020C046C0461E
:1098000002BD01468008081A02091018020A101841
:10981000020C1018C008820012185200891A01E0C8
:10982000401C0A390A29FBD27047000010B500F02D
:1098300017FC001D10BD00BFC55F000010B503463A
:10984000406801E003464068002801D08842F9D30F
:109850001868C3188B4206D0CB1CD808C000001D66
:10986000411A521A0146081D0A60FEF7ECFD10BDB0
:109870000B4670B5024689078008084319469D08C3
:10988000141AA94125090807054308092C1948415C
:10989000250A01060D43010A2C194141200C0D0433
:1098A00028430D0C00194D41002140194D41C008BD
:1098B00069070843E908840F8D00254384002418B4
:1098C0004D4124196D41121BAB4107E00925ED43C1
:1098D0002C11521963410024401C61411C460A2589
:1098E0000026551BB441F1D270BD0000FFB50C46F7
:1098F0001E468FB003CA089009914F007D0D00D11C
:109900006D1E002108460020C0460321099A8905E2
:109910000840002A03DA8200801840080840800DC1
:1099200001280A9002DD0020C0430A9008980743EE
:109930000DD0F048F049281848430714189800281B
:109940001DD07542291E1DDD0A9842421BE0189861
:10995000012802D00020302104E00020F24305E07D
:109960002154401CB042FBDB30460022189B0021F2
:1099700021540F998B600A60486013B0F0BDBD1B85
:109980006D1CDFE70A9A002900DA69420BA800F093
:10999000AFFB0BAB07CB03AB07C30899099800F0EB
:1099A00013FC6B4607C30146D4480918002D0091EB
:1099B0000BDDD24903980A9A49424018002303A9B3
:1099C0000390684600F070FE08E003990A9A0023AD
:1099D000081803A90390684600F010FE6B4607C301
:1099E0000004000C03D00020C043410800E01046F2
:1099F000189A002A03D00022009215461EE0751E18
:109A000005D4FFF735FF303262556D1EF9D50122BE
:109A10000843079602D000227F1C04E020783028FB
:109A200001D100227F1E002A069787D01EE0112D4B
:109A300007DAFFF71DFF303262556D1C02460A43FC
:109A4000F5D1084303D00098002819D00EE000217A
:109A5000681E05E0235C625C63542254401E491C6E
:109A60008142F7DBA81B401E07950690079A1899BC
:109A70000020A0540F98079B069A81600CC07CE7D9
:109A800011260020189059E7D21DF0B50D46044666
:109A9000D10893B0C90003C90C900D9105F082FE66
:109AA00002460D98C00F01D02D2007E020688107E5
:109AB00001D52B2002E04007C00F4001032A0F9080
:109AC00001D0072A05DB03462946204600F0CCFAE0
:109AD0000EE12078800601D5E76900E006272846D8
:109AE000652D04D0662814D0672D69D12DE00020A3
:109AF000112F009001DB112300E07B1C0CAA03A9AD
:109B000010A8FFF7F3FE1199002610987D1C0E9106
:109B100042E001203B460CAAC0070B9001200090B8
:109B200003A910A8FFF7E2FE119D129810990026D4
:109B300000280E9501D1781C0D18781B02D44642DE
:109B40007D1C761EE81B00903AE0012F00DA012709
:109B50000020112F009001DD112300E03B460CAAEC
:109B600003A910A8FFF7C2FE11993D4610980026E0
:109B70000E91217809070BD40E99A94200DA0D46FF
:109B800003A9012D04DD4A19203AD27F302A06D0DC
:109B9000B84201DA011D04DA012100910FE06D1EC7
:109BA000EFE7002802DC86192D1A03E0411CA942C8
:109BB00000DD0D46801B401C00900120C0070B906B
:109BC0002078000705D40098A84202DB0020C0439B
:109BD000009069460020C8720B98012102AF03373C
:109BE000C907884225D0022010902B2011900B9895
:109BF00000280BDA40420B902D20119006E00B98C4
:109C0000FFF7FFFD30317F1E0B9039701099481E11
:109C100000291090F3DC0B980028F0D111987F1EDA
:109C200038702088000501D5452000E065207F1EA2
:109C3000387001A8C01BC01D0B900F98002800D0E1
:109C4000012041190098C01709180B980818A1693C
:109C5000081A401EA0612078C00602D42046FEF7F4
:109C6000F5FC0F98002805D06268A1689047206A2B
:109C7000401C20622078C00625D52046FEF7E6FC71
:109C800021E0002E07DB0E98B04204DD03A86268D5
:109C9000805DA16802E06268A16830209047206A78
:109CA000761C401C20620098401E002800900AD1BB
:109CB00000F0D6F9C06862680168405CA16890470E
:109CC000206A401C206228466D1E0028D9DC07E06F
:109CD00062683878A1687F1C9047206A401C206227
:109CE0000B99481E00290B90F2DC2046FEF7C4FCBD
:109CF000032042E601FCFFFF104D0000E1DFFFFF03
:109D0000D21DF0B504460D46D0088DB0C00046689F
:109D100007683146384605F045FD0246F00F01D090
:109D20002D2307E02068810701D52B2302E040079F
:109D3000C00F43016846002B037001D0012000E0F2
:109D40000020032A0A9001D0072A04DB2946204676
:109D500000F08AF92DE12078800601D40D2500E07D
:109D6000E5697000400D0D2D01904BDA300D00219A
:109D70000B9008460020C046032189050840002EAC
:109D800005DA82008018C20F1018401008408015B4
:109D9000012801DD0020C043A9000023182906D3B3
:109DA0009C460A460123183A1B07D34003E00122D0
:109DB0001205CA4094460C31202902D33A46203974
:109DC00000E032468A40002802DD002A06D119E070
:109DD000002817D10121C9078A4213D319466346C7
:109DE0007F185E41002806D10120C007824202D1BF
:109DF000084687439E430B98310D814202D001985B
:109E0000401C01902088000502D57149794402E088
:109E10006F49794419396B460A9830221A540A98C6
:109E20000A7C401C1A54401C0A900198002801DC4E
:109E3000302000E031201872019A0120002A02D05F
:109E4000644BD21804E072003A4302D0614A521CBB
:109E50000192002D02DC2278120703D56A462E20DB
:109E6000507202200022864694460CE032033601EE
:109E7000120F6D1E8B5C02AA13546246521C401CCA
:109E80009446052A01DA002DF0DC002202AE08E03B
:109E90003B0F3F01CB5C521C6D1E3354401C082A03
:109EA00001DA002DF4DC23689A0601D511E0401E8A
:109EB000704504DD3218203AD27F302AF7D00028CE
:109EC00007DD3218203AD27F2E2A02D11A0700D499
:109ED000401E002D03DD3E223254401C6D1E497C85
:109EE00031540199401C002906DA2D21471C3154B8
:109EF00001984042019003E02B21471C3154019806
:109F00007D21C900884206DBFFF7D8FB3030F055D1
:109F10007F1C019101E0642808DB01986421FFF7B0
:109F2000CDFB3030F0557F1C019101E00A2806DBA3
:109F300001980A21FFF7C2FB3030F0557F1C0198D1
:109F40000A21FFF7BBFB3031F1550A98A1697F1C4C
:109F50007A191018081AA0612078C00602D4204689
:109F6000FEF774FB216A6E460A980818206204E026
:109F700062683078A168761C90470A98401E0A9063
:109F8000401CF5D12078C00602D52046FEF75EFBC6
:109F900002AE09E03078761C3E280DD06268A168D8
:109FA0009047206A401C20627F1EF3D22046FEF7B5
:109FB00063FB0DB00320F0BD206A4019206203E06E
:109FC0006268A168302090476D1EEDD3F8E700006D
:109FD000BB5A000001FCFFFF10B54369002B02D003
:109FE000C046C04601E0FFF737F8012010BD1288D7
:109FF0000146243182840022C2840122ECE71168E8
:10A000000022D243E8E7F8B516460C460546FFF7AE
:10A010000DFC0368FF200230C05C012807D0FF2C34
:10A020000FD8185D00280CD001202C70F8BDFF332C
:10A030003246214608331868C71828460023B84717
:10A04000F8BD0020C043F8BD10B500F083FB00F060
:10A050007BFB10BD10B500F097FB00F075FB10BD49
:10A060000048704748D40030F8B51F460446012325
:10A070000068DB02032601461840072A05DB00289A
:10A0800001D017A506E017A504E0002801D016A509
:10A0900000E016A5102081432160A069C01E002F9A
:10A0A000A06101D0401EA0612046FEF7CFFA002F2C
:10A0B00009D038466268A1689047206A401C206237
:10A0C000C01C206206E0206AFAE762682878A1686E
:10A0D0006D1C9047761EF8D22046FEF7CDFAF8BDEB
:10A0E0004E414E006E616E00494E4600696E66003C
:10A0F000F7B516468AB0334878446C4603467C333D
:10A10000C06F5A689B680DC42E487844763003AC03
:10A110000DC80DC43720C001081837211B30FFF7C8
:10A12000CDFA05460C46803D1B3C02D56442012019
:10A1300000E000200027099010E0E0070CD00C2080
:10A1400020497843794432464C3941186846012306
:10A1500000F054FA6B4607C364107F1C002CECD14E
:10A16000184F7F442E3F16E0E80712D02001C01997
:10A170000EC80691089307920068F04201D1981921
:10A1800008903246012306A903A800F037FA03AB72
:10A1900007C36D10641C002DE6D10998002806D075
:10A1A00032466946012303A800F07EFA05E0012348
:10A1B0003246694603A800F021FA0A9B07C30DB096
:10A1C000F0BD0000E4570000034640000A4610B509
:10A1D000400D0BD00121C9070F24A40200191C0354
:10A1E00064082143540D2143D20207E000210120DD
:10A1F000F2E7D40F490021435200401E0029F8DA4B
:10A20000DB0FDB07184310BDFFB50D46144685B0C4
:10A210004868516805F0ACFA00910190A868A168FF
:10A2200005F0A6FA02910390A868616805F0A0FA0B
:10A23000029A12188242029201D2012000E000200C
:10A24000019A0B18D2180028019202D08A4202D932
:10A2500003E08A4201D2012000E0002000990818A2
:10A2600000906868A16805F083FA029A1218824289
:10A27000029201D2012000E00020019A0B18D218AE
:10A280000028019202D08A4202D903E08A4201D218
:10A29000012000E00020009908180090286821683B
:10A2A00040004900400849084018FA49471814E09E
:10A2B00001994000C90F084300900198029940009D
:10A2C000C90F08430190029803994000C90F084341
:10A2D0000290039840007F1E039000980028E7DA60
:10A2E0000898002801D0EC4E00E00026B74201DAC1
:10A2F000012000E00020002804902AD0F71BF80677
:10A30000C00E15D0029B2021091A039A8B401A43D4
:10A310000392029A019BC2408B401A430292019A17
:10A32000009BC2408B4000991A430192C1400091AA
:10A330007B110DD06F460320C11A03D50021820086
:10A34000B95003E08A008100BA587A50401EF3D514
:10A35000374603980299002800D00120014308984D
:10A360000291002808460CD0002800D00120019955
:10A37000019A490508430121D20AC902D202019279
:10A3800000E001210E9B0122D207012B02D0002BFD
:10A3900003D013E0002807D120E0904204D8904277
:10A3A0000CD1019B0B4209D0019B5918019105D199
:10A3B0000099491C009101D17F1C009200280DD00A
:10A3C000102108460020C0460498002806D00F98A7
:10A3D000002803D0082108460020C04628682168CC
:10A3E000019B009A4840C10F0598C90739430EC028
:10A3F00009B0F0BDFFB587B0099A0898089953686D
:10A4000092684068896896460022039317469446EE
:10A41000089A12685300099A5B08126852005208A1
:10A420009A1A9E4BD4180A9A002A01D0352200E0CD
:10A43000402206920022012315460492DB07059371
:10A4400024E0002D05D175460346039E4D1BB34104
:10A4500009D375466646039B491B049D9841059B9D
:10A460007519AC465F4163463B4308D0059B049E8B
:10A47000DD0776082E435B080496059301E0521E23
:10A48000641EC50FED0749184041521C069B9A42B5
:10A49000D7DB002D04D17546039A6B1A824101D295
:10A4A00003200CE0039A0B466B404240134303D059
:10A4B000014303D0012002E0022000E000206146B9
:10A4C00001910021009702910A99002905D0614667
:10A4D00040020143704B019102E08007002302908B
:10A4E0009C4201DA012000E0002007003AD01A1B4C
:10A4F000D006C00E15D0029D2021019C091AC5402E
:10A500008C402543029C8C4000D001242543019CB3
:10A510000295009DC4408D4000992C430194C14098
:10A52000009154111DD06D460221002202290CD148
:10A530000320001B07E0002804DB8600AE59002E34
:10A5400000D00122401C0328F5DB081B02D588003F
:10A550002A5004E08000285810438A00A850491E61
:10A56000E3D51C460A98002802980CD0002800D099
:10A5700001200199019A490508430121D20AC90223
:10A58000D202019200E00121109B0122D207012B8F
:10A5900002D0002B03D013E0002807D11FE0904227
:10A5A00004D890420CD1019B0B4209D0019B591851
:10A5B000019105D10099491C009101D1641C0092C0
:10A5C00000280CD0102108460020C046002F06D0DD
:10A5D0001198002803D0082108460020C04608989A
:10A5E0000999019A009B006809684840C10F0798C3
:10A5F000C907214382600AC00BB0F0BD00B585B029
:10A60000019300920A460146002302A8FFF7FCFDD1
:10A6100002A807C805B000BDFFB50A461F4685B0B1
:10A620000799019301230091014602A8FFF7ECFD71
:10A6300002990398049ECA0F4900D20700920F2284
:10A64000490892028C1A0021002800DB0C464500C4
:10A6500013486D08844214D3079A002A04DA441E72
:10A660000026104DF64302E004460D460E4610212A
:10A6700008460020C046002F03D0042108460020D1
:10A68000C0462005E90A0843009908436905F20A13
:10A690001143ADE602C0FFFF013C0000FF3F000098
:10A6A000FF070000FFFFFF7F00B585B00193009218
:10A6B0000A460146002302A8FFF79CFE02A807C82D
:10A6C000A8E7FFB50A461F4685B007990193012305
:10A6D0000091014602A8FFF78DFE02990398049E9F
:10A6E000CA0F4900D20700920F22490892028C1A21
:10A6F0000021002800DB0C46450011486D0884420B
:10A7000014D3079A002A04DA441E00260D4DF6439E
:10A7100002E004460D460E46102108460020C046C1
:10A72000002F03D0042108460020C0462005E90A76
:10A730000843009908436905F20A114358E60000EE
:10A74000FF070000FFFFFF7F10B5002801D002F0D7
:10A7500057FF10BD10B5014602A000F03DF80120E2
:10A7600010BD000053494752545245443A205265A7
:10A770006469726563743A2063616E2774206F7038
:10A78000656E3A200000000010B5012805D00021B8
:10A7900003A000F021F8012010BD09A1F8E7000096
:10A7A00053494752544D454D3A204F7574206F66BA
:10A7B0002068656170206D656D6F72790000000022
:10A7C0003A2048656170206D656D6F727920636F06
:10A7D000727275707465640070B505460C460A2087
:10A7E00000E06D1C02F086FF002D06D028780028BE
:10A7F000F7D102E0641C02F07DFF002C02D020782B
:10A800000028F7D10A2002F075FF70BD70B58C18D2
:10A810000578401C6B075B0F01D10378401C2A119F
:10A8200006D10278401C03E00678401C0E70491CDB
:10A830005B1EF9D12B0705D40023521E0DD40B70DB
:10A84000491CFAE70378401CCB1A921C03E01D78E0
:10A850000D70491C5B1C521EF9D5A142D8D30020B3
:10A8600070BD00000549064A8A42104600D10548DD
:10A870008A4200D10449FDF76CBDC0460000043097
:10A88000101B0130081B013000C0003080B503F000
:10A8900003FE80BC01BC864603F076BC80B500F0A8
:10A8A000DDF800B180BD80BC01BC864600F04EB82A
:10A8B000B0B542684B689A420CD16AB18968836826
:10A8C00000201C780D78654028435B1C491C521EF3
:10A8D000F7D102E00120B0BD002041420143C80F82
:10A8E000B0BD0000F0B503AF83B06E4629B1716012
:10A8F00028B10023DA4302250AE0022521E0384886
:10A9000000683849B1FBF0F14A1C424300231D4660
:10A9100035480068C11D0724A1436C46B4606C46ED
:10A92000641AA54682B069460860204602F002FF1C
:10A9300002B020B92046716803F00AF80546B068F5
:10A9400085462846FC1F053CA546F0BDB0B502F083
:10A95000EBFE044602F0E0FE244D286002F0D4FE37
:10A960001F490860286840F22711B1FBF0F1491C2B
:10A9700041431D4801602046B0BDC046F0B583B0DC
:10A98000022452B30346906838B3002513B1EB4359
:10A99000022407E0124B1C68124BB3FBF4F35B1C60
:10A9A000634300245768104E36686FB10F4D029311
:10A9B00033462E687D1EB5FBF6F56D1C75431E46AD
:10A9C000029B1268954208D86A46156059188A1980
:10A9D000002302F0AFFE00B90446204603B0F0BDEC
:10A9E000801A0130FFFFFF03781A01307C1A013012
:10A9F000F0B5A1B050B3044600201F901E901EA8D1
:10AA0000144E0822314602F09BFF0425F8B91EAF10
:10AA1000384603F022F80190381D03F01EF8022892
:10AA200015D102A87021FEF79AF904250A48019968
:10AA300081420CD102A87022314602F081FF30B968
:10AA400002A8214602F0DAFF054600E0022528466A
:10AA500021B0F0BD00A00210D4B3515A02F02CBFB7
:10AA6000F0B5BFB05A4C002800D18BE08768002FAA
:10AA700000D187E00E46002900D183E04568402DD3
:10AA800000D97FE0002A00D17CE0B068002800D126
:10AA900078E09068002875D01068202872D3019261
:10AAA0002FA84021039136220292FEF731F91FA808
:10AAB0005C2203990392FEF72BF9FDB138780299D5
:10AAC00048402FA908703878039948401FA908709A
:10AAD000012D13D0681E1FA9491C7A1C2FAB5B1CCB
:10AAE0001D7817786F400D781F7017786F400F70C2
:10AAF000401E491C521C5B1C0028F1D104AF384693
:10AB000003F06EFE0021384603F09EFE70BB04A8E1
:10AB10002FA9402203F0E8FE40BB7268B16804A888
:10AB200003F0E2FE10BB0198816804A803F0C4FDA5
:10AB3000E0B904A80026314603F086FEB0B904A8A7
:10AB40001FA9402203F0D0FE80B90198816804A8B3
:10AB500020273A4603F0C8FE40B90198816804A84E
:10AB600003F0AAFD10B901984760344604A803F029
:10AB700032FE2FA84025294603F092FD1FA8294642
:10AB800003F08EFD20463FB0F0BDC04670B584B0E6
:10AB9000044601680E4D202910D3A06803F076FB0F
:10ABA00060B90C4801A90A4668C868C210206060F4
:10ABB00020462246FFF754FF054630B12168A068C1
:10ABC000FEF7CBF8284604B070BD0025FAE7C04672
:10ABD0000100435574F90110FEE7F0B582B001920F
:10ABE00000230124032200921E462746B7400F424D
:10ABF00007D0019F9F40009D9D400268AA433A43B1
:10AC000002609B1C761C102EEFD102B0F0BDF0B597
:10AC100082B0019200230124032200921E4627469F
:10AC2000B7400F4207D0019F9F40009D9D40026B9F
:10AC3000AA433A4302639B1C761C102EEFD102B04C
:10AC4000F0BD4AF64D40C1F20100004700F09EFE03
:10AC5000FDF7DEFAFEE7FEE710B50146134A83581A
:10AC600001205B0007D5124A8958C90309D5F84964
:10AC70000020087210BD8A18830712681A4203D098
:10AC800010BDF349087210BD40F620028858802399
:10AC90001843885006480858012424040440200C16
:10ACA000EB4C20728C589C438C5010BD280800003F
:10ACB0002C080000F0B585B00446E54E7268092105
:10ACC00001AB00F081FB3068C11E4E4D0198012997
:10ACD00039D8800F032850D37268072100252046F9
:10ACE0002B4600F017FB40F20840474F27504748DB
:10ACF00044492150082120462A4600F09FFB0028A5
:10AD00007DD107210022204600F0C8FB40F620003C
:10AD1000215840220A432250201801684906FCD4D9
:10AD2000D42038587072410E3174410CF173410ACD
:10AD3000B17341087173010E3173010CF172000A95
:10AD4000B072304D54E0800F029834D001A9498987
:10AD50008006800A081840024019401C7073010EDA
:10AD60003174010CF173010AB173C10D3173C10B60
:10AD7000F172C109B172400039E0002030743073C3
:10AD800003988103490F04228A40800F02998B05A2
:10AD90001B0D1818401C50430903090F8840810EF1
:10ADA000F173810CB173810A7173410EF172410C20
:10ADB000B172400A1BE000213174317303998A0398
:10ADC000520F04239340890F8205120D8918491CE4
:10ADD00059430003000F8140880EF073880CB07354
:10ADE000880A7073480EF072480CB072480A70728C
:10ADF00000203075F074681C7074000AB07405B0DF
:10AE0000F0BDC046FF01000080D4003038080000CB
:10AE1000F0B58BB0064640F2001740F200112C311D
:10AE200000F03AFC40F62000315820220A4332500C
:10AE30003018C94C217A0268920603D50029FAD14C
:10AE4000C44D02E1002130460A4600F027FB41F2E2
:10AE5000000001E00A98401E0A900A980028F9D1E3
:10AE60007C48012505707C480490049B40F2001248
:10AE700055320821304600F04DFA0A900A98002811
:10AE8000029534D0002130460A4600F007FB0A97AD
:10AE900002E00A98401E0A900A980028F9D1049B03
:10AEA0003721002530462A4600F034FA0A900A98E5
:10AEB00002284ED13046002603903146324600F03B
:10AEC000EDFA0A9702E00A98401E0A900A980028B4
:10AED000F9D1624D02992970049B624A039800F0EF
:10AEE00019FA02283ED126609A48451CADE0049B21
:10AEF00037210022304600F00DFA58480570049BB7
:10AF00002921584A304600F005FA40F630017058C1
:10AF1000020218D4701803900298C4053727002540
:10AF2000049B304639462A4600F0F4F901204B498B
:10AF30000870049B292130464A4A00F0EBF9039837
:10AF400000682042ECD0400209D5029D2A46EB4C15
:10AF500053E00A9808B32560E748451D75E00222D2
:10AF6000E64C49E040F63001039840580202029F47
:10AF70003C4C0ED4039840180190FE052F70049BA2
:10AF800003983946224600F0C5F90198006830421E
:10AF9000F4D040022DD504222CE03048029D0570EB
:10AFA000049B29212E4A304600F0B4F940F63000C7
:10AFB00031580222090220D4019230180390EC0586
:10AFC00037250027049B304629463A4600F0A2F96F
:10AFD000029822490870049B29213046204A00F03B
:10AFE00099F9039800682042ECD0F34C029D019A35
:10AFF00003E00322F04C039E029D22600221002206
:10B0000005AB304600F0E0F92068C01E01280BD8DF
:10B0100030462E040321002532462B4600F07AF9F3
:10B02000099050B9666010E00321002530462A4699
:10B030002B4600F06FF9099008B1099D05E040F634
:10B0400030003058000A0004606028460BB0F0BDA4
:10B050005CD4003074D40030FFFF0F00341A01308C
:10B060000080FF000080FF40F0B581B000910446F1
:10B0700040F2004002272750201840F600016618D1
:10B0800001688907FCD40125056003203060306821
:10B09000C007FCD1E8481521FDF761FE37600C4878
:10B0A0002158AA07009B9B0501D5914300E011435D
:10B0B0002150215840F200120A432250316A44F2D2
:10B0C000000001433162316A0142FCD101B0F0BDA0
:10B0D0002808000010B504461D480021215040F604
:10B0E000200021580F221206914321502158092295
:10B0F00012060A4322502158FF2212049143215084
:10B100002158012212040A432250215848F2000219
:10B11000914321502046FFF79FFD20B12046FFF7C5
:10B1200077FE10B110BDEF4810BDED480068032850
:10B1300001D10B4900E0094900F0AEFA2046FFF7C3
:10B14000B9FD204610BC02BC8E4600F0CDB9C04609
:10B15000040800001001FFFF5CD40030A86100006B
:10B16000204E0000F0B58BB0044600200A90DD4868
:10B1700073B11E4617460691D9484268072100253B
:10B1800020462B4600F0C6F8079018B10798B1E0AA
:10B19000C01CAFE0049540F620000594241840251B
:10B1A00020682843206020684006FCD4E068000640
:10B1B000F6D553485349059A1150C94800680128EB
:10B1C00002D0042800D07F02069AC34805990F5088
:10B1D00040F208400A50FF2006900296B6FBF0F0BD
:10B1E00003900890089A7AB3BD48027A4649474FBF
:10B1F00006980604012001900498387023680B40DB
:10B200000993099B334309930A98099B18B10420B9
:10B210000343236004E03E480343236001980A90FF
:10B22000387820B9387810B9002AF9D137E0E068C9
:10B23000400747D5E068000739D50898401E0890B8
:10B24000089800283049D7D1069B039858430299A3
:10B25000081A0890089868B32C4904980870206868
:10B2600043F60072904309901804099A82430992A8
:10B2700008980004099A024309920A9A09981AB197
:10B2800004221043206004E0214A10432060012082
:10B290000A909348007A0A781AB90028FBD191489D
:10B2A00028E0E06840070DD5E068000702D48D482B
:10B2B000C01D1FE00C21002605983246334600F0E1
:10B2C00029F810B18748801D14E0206828432060C9
:10B2D00020684006FCD4E0680006F6D507210598F2
:10B2E000324600F0DBF820682843206020684006E2
:10B2F000FCD430460BB0F0BD1001FFFF5CD4003031
:10B3000038080000FF010000FFC0FFFF351A0130C0
:10B3100007120000B0B5704C025140F6200284586C
:10B32000244D254009022943C91C81508118D74A60
:10B33000127A43B1DB430C68A4070BD55B1C22D007
:10B34000002AF8D104E00B689B0703D5002AFAD144
:10B3500064492CE019490A78012A0BD1184A82580D
:10B36000D2B2552A06D040F6300282580F2313403D
:10B37000012B18D1134A117861B100211170464A8E
:10B380000223835013E0086844F2000202430A607B
:10B3900002210CE040494058400701D50020B0BDD3
:10B3A0005048801DB0BD002008704E490931084644
:10B3B000B0BDC046FCC0FFFF5CD4003074D4003088
:10B3C00034080000341A013070B585B0424C025187
:10B3D00040F620028458174D2540090229431131B7
:10B3E00081508118A94A127A0C68E40603D5002A14
:10B3F000FAD13C481CE028494158490702D4394851
:10B40000801D15E00021425812BA6C466250091D99
:10B410001429F8D16846011D0020009C02468D5871
:10B420002E0E240234199C50121D102A2C46F6D1DF
:10B4300005B070BDEEC0FFFF5CD4003010B5264BE8
:10B44000C25040F620028358124C1C40090221438E
:10B45000C91D815081188D4A127A0B689B0702D54D
:10B46000002AFAD104E00B685B0703D5002AFAD161
:10B470001C4810BD084A815849071A4901D4881D43
:10B4800010BD80180068000701D5002010BDC81D40
:10B4900010BDC046F8C0FFFF2C08000010B581B0F9
:10B4A000002300930C4BC25040F6200283580B4CF3
:10B4B0001C4009022143491C81508158C90708D00A
:10B4C00080187249097A074A01B900920368DB07BC
:10B4D000FAD1009801B010BD24080000FEC0FFFFA3
:10B4E0005CD400301001FFFFF0B583B0044667481C
:10B4F000426800230293072520462946FFF70AFFEA
:10B50000029018B1029D284603B0F0BD40F2004001
:10B510002146241840F6200001910E18402730687B
:10B520003843306030684006FCD4F0680006F6D539
:10B5300056480068401E032800D987E0810001A218
:10B5400051188F4600F006B800F036B800F061B828
:10B5500000F064B840F208409349019A1150F7484E
:10B560001550F54845683721002310462A46FFF755
:10B57000D1FE02900028C5D18B4D206802210143E5
:10B58000216020688007FCD433210022019C2046E2
:10B59000FFF754FF02900028B4D128780F21014012
:10B5A0000F2922D1204600F0BDF802900298E0B9A0
:10B5B0005B4900F071F818E040F208407A49019CBC
:10B5C0002150DE482550DC484268372100232046C0
:10B5D000FFF7A0FE0290002894D1332100222046DC
:10B5E000FFF72CFF029000288CD1D3484268372106
:10B5F00000232046FFF78EFE0290002800D081E74E
:10B600000621022200232046FFF784FE0290C0B1EB
:10B6100078E7306848F200018843306006211C4A10
:10B6200000230198FFF776FE0290002800D069E71A
:10B6300030683843306030684006FCD4F06800065B
:10B64000F6D5306848F2000101433160BC4D6A1CF8
:10B6500010210023019C2046FFF75CFE0290002889
:10B6600000D04FE7B54825500721002520462A463F
:10B67000FFF714FF30683843306030684006FCD470
:10B680000448215801220A4322503CE75CD4003090
:10B690000001B70328080000B0B50C4601F058FFC0
:10B6A000C00038D41C4D2846103800688002800F36
:10B6B000012805D0022806D0032807D117480BE03F
:10B6C00003F0C6FF04E003F0C9FF01E003F0CCFF84
:10B6D00040F2E831B0FBF1F011498C4200D30C4646
:10B6E000B0FBF4F14C43001B00D0491C40F20010A9
:10B6F000FF2902D80029084604D0FF2109060006C8
:10B70000401800E00020FF2109062A688A432A60C9
:10B71000296801432960B0BD20020040E02E0000EE
:10B7200050C30000F0B581B004460020009040F204
:10B7300008401D4E2650814D3F27675106211B4A68
:10B740002046FFF77BFE0090012310B1184601B0A0
:10B75000F0BD40F208427078317809020818F5D03F
:10B76000707F317F09020818F0D16019A1180E60AE
:10B77000076006210E4A20461D46FFF75FFE2B4656
:10B7800000900028E2D140F62000215840220A43D0
:10B790002250201801684906FCD4707831780902DB
:10B7A000081843424341D1E780D4003001FFFF0035
:10B7B00001FFFF80F0B58BB0044600200A905D4881
:10B7C00073B11E46154606915B4842680721002763
:10B7D00020463B46FFF79EFD079018B107987BE097
:10B7E000C01C79E0049740F62000059424184027F7
:10B7F00020683843206020684006FCD4E0680006DA
:10B80000F6D54E484E49059A11504B48006801281C
:10B8100002D0042800D06D024A4805990D5040F22C
:10B820000840069A0A50FF2006900296B6FBF0F1F7
:10B8300003910891089A52B33F490A7A4248434D0E
:10B8400006990E040121019104992970236803408F
:10B850000993099B334309930A99099B19B108215C
:10B860000B43236004E03A490B43236001990A919A
:10B87000297811B9002AFBD12DE0E168890753D45A
:10B880000899491E0891089900292F48DCD103998D
:10B89000069848430299081A0890089808B32B485C
:10B8A0000499017008992268274B13400904194331
:10B8B00009910A9A09991AB108221143216004E0FA
:10B8C000234A1143216001210A911B49097A027818
:10B8D00022B90029FBD117480BB0F0BDE068800702
:10B8E00022D40220E0600C21002505982A462B4630
:10B8F000FFF710FD10B10F48801DEDE720683843B9
:10B90000206020684006FCD4E0680006F6D50721D8
:10B9100005982A46FFF7C2FD20683843206020685A
:10B920004006FCD42846D7E70220E06001480830F2
:10B93000D2E7C0461001FFFF5CD400303808000099
:10B94000FF0100002408000080C000FF351A01300C
:10B950000B19000080B503F07BFE0749086003F077
:10B9600089FE06490860064940180649B0FBF1F017
:10B970000549086080BDC0464CD2003050D200302E
:10B9800020A1070040420F0048D2003010B501F05E
:10B99000DFFDC00013D40C48592116228823016012
:10B9A000026003600468002CF9D00021CA43074BF1
:10B9B0001A60243801601869054901431961054876
:10B9C0000549016010BDC04600010040F40100407F
:10B9D0000040F0FF08ED00E000800110B0B5044623
:10B9E000204DA8420ED0002020498C420CDD204979
:10B9F0008C4211D01F498C4210D01F498C421ED15D
:10BA000020480EE016480CE01C498C4208D01C4926
:10BA10008C4214D11E4804E01C4802E01A4800E0A1
:10BA2000114803F02DFE022806D12248844207DC8B
:10BA3000AC420BD0114807E0800016A10858B0BDF9
:10BA40000D48844202D00B48844204D1B0BC01BCF2
:10BA5000864603F01BBEB0BC01BC864603F01CBE8C
:10BA60000200805E000005400300C05EFF1005502C
:10BA7000001105500020055000210550000105402F
:10BA8000001005500500C0BE040080BE0500405FE8
:10BA90000400005F001BB7000080000000000000F1
:10BAA0000000000000093D00007D000000000000D3
:10BAB000001BB700FF1F0550F0B589B00D460446C6
:10BAC000834801A9CCC8CCC1CCC8CCC18148844230
:10BAD0000ADC8848844215DC8A48844225D08A489A
:10BAE000844224D0894809E07B48844212DC7E48A5
:10BAF00084421AD07D48844219D07D4884425CD16A
:10BB0000864E25E07C48844213D07C4884421ED077
:10BB10007B4806E0714884420BD07148844216D0BD
:10BB20007048844249D17A4E04E07E4E10E07C4E4B
:10BB300000E0794E304603F0A3FD0746304603F09F
:10BB4000B1FD0090042F11D103F0A6FD0CE0714E61
:10BB5000304603F095FD0746304603F0A3FD009004
:10BB6000042F03D103F092FD0590042700202063E9
:10BB70000326E660A06812490140A160012F02D1AE
:10BB800003F066FD0290C5B1B80001A908580099FC
:10BB9000491CB0FBF1F069084118B1FBF5F1891EB1
:10BBA0000A0C07D0E9004018B0FBF5F00009801E30
:10BBB000606202E030070143616209B0F0BDC04637
:10BBC0000FFFF0FFF0B58BB0019302920C460546D3
:10BBD0003F4803A9CCC8CCC1CCC8CCC13D488542A4
:10BBE0000ADC4448854215DC4648854225D0464853
:10BBF000854224D0454809E03748854212DC3A485E
:10BC000085421AD03948854219D0394885425DD1DC
:10BC1000424F26E03848854213D0384885421FD02D
:10BC2000374806E02D4885420BD02D48854217D075
:10BC30002C4885424AD1364F04E03A4F11E0384F44
:10BC400000E0354F384603F01BFD0646384603F04A
:10BC500029FD0746042E12D1042603F01DFD13E032
:10BC60002C4F384603F00CFD0646384603F01AFD0B
:10BC70000746042E03D1042603F008FD04E0012E3C
:10BC800005D1012603F0E4FCB10003AA505010983E
:10BC9000BCB1B10003AA51587A1CB1FBF2F26108A1
:10BCA0005118B1FBF4F1891E0B0C06D0E1005118BC
:10BCB000B1FBF4F10909891E02E0032212071143C6
:10BCC00069620299019A0A430243EA600BB0F0BD2F
:10BCD000E4050210FFFF0650FF2F07500030075009
:10BCE0000040075000500750000007500010075058
:10BCF00000200750FF2F074000300740004007405A
:10BD00000050074000000740001007400020074097
:10BD1000953DCC7F143D8C7F933CCC6F123C8C6F57
:10BD2000913D406F103D006F80B501F093F80149DF
:10BD3000086080BD9CD9003080B501F0BDFD414256
:10BD4000484180BD01F0ACBDF0B581B004461B4E4A
:10BD5000354670353746384601F0AAFDC719AF425F
:10BD6000F9D3174DAF4209D216A001F0C3FE244803
:10BD70003918304601F06EFDD8B903E040F20040BA
:10BD8000241835462F19AF4209D92E46304601F006
:10BD90008FFD8619BE42F9D31A48864204D8284638
:10BDA000214601F057FD04E0174801F0A3FE0020F2
:10BDB000C04341424141084601B0F0BD00A002101D
:10BDC00000A402105B444247205D20457261736904
:10BDD0006E67206865616465722073657061726169
:10BDE00074656C792066726F6D2061637469766525
:10BDF000206170706C69636174696F6E0D0A000078
:10BE00000060FDEF00001010410A0210F0B587B08D
:10BE100079B10C46054601F047FD06463349B1FBB2
:10BE2000F0F07043081A06D0314801F063FE30BFCD
:10BE3000FDE7002022E02F4806900021059144F202
:10BE40000000B0FBF6F070430490A768E2683B4640
:10BE5000134393B10394C31B0B46934100D338465D
:10BE600005902548836904AA28460091984738B16F
:10BE700022A001F03FFE009800E0012007B0F0BDD5
:10BE8000039808300390701E0290002701970598D0
:10BE90000028EDD02C4615497918029A1018B0FBED
:10BEA000F6F5754306982A4601F00AFD0146404220
:10BEB0004841EF19039A13685268FD1A019D954194
:10BEC000DCD20029DAD10025D81BAA4104990B1A2B
:10BED000954100D3014605910748836904AA254688
:10BEE0002046394698470028D1D0C1E700A4021067
:10BEF000310A0210B0D900301CD200305B444247F6
:10BF0000205D2041524D5F5543505F526561642072
:10BF100072657475726E6564203020627974657321
:10BF20000D0A000070B50C46064610A001F0E2FDB7
:10BF3000A068FFF709FF0025B0B115A001F0DAFDF8
:10BF4000204600F023F978B117A001F0D3FD304668
:10BF50002146FFF75BFF38B11AA001F0CBFD204668
:10BF600000F03EF845424541284670BD5B444247DB
:10BF7000205D204572617365206163746976652078
:10BF80006170706C69636174696F6E0D0A00000006
:10BF90005B444247205D2057726974652068656183
:10BFA0006465720D0A0000005B444247205D204337
:10BFB0006F7079206170706C69636174696F6E0D68
:10BFC0000A0000005B444247205D205665726966A6
:10BFD00079206170706C69636174696F6E0D0A001D
:10BFE000F0B5A5B0012528B104465D48016A204698
:10BFF000884710B1284625B0F0BDA068E16801432C
:10C0000000293FD0009408340AAD284602F0E8FB2E
:10C010000021284602F0EAFB02A82021FCF79FFE3F
:10C0200001942068E0B1814D064603E0361B17D02D
:10C030000198006844F200018E42344601D344F274
:10C0400000041249891B09182846224601F078FC91
:10C0500007460AA82946224602F044FC002FE5D0F4
:10C060000AAD02AE2846314602F024FB284602F013
:10C07000B2FB0098103020223146FCF7A1FD18B920
:10C080000546B7E70225B5E70125B3E700A402108E
:10C09000F0B59FB0D1B30F46054630481CA91CC867
:10C0A0001CC101AE304602F09BFB0021304602F07D
:10C0B0009DFBB8680097F96802460A439AB1820B63
:10C0C0008B04D218890B114309B144F200001D9072
:10C0D0002348836900261CAA284631469847C0B1E8
:10C0E00020A001F007FD01AD504E2846314602F078
:10C0F000E1FA284602F06FFB00981030202231460A
:10C10000FCF75EFD01464042484100E000201FB0C0
:10C11000F0BD009C083437461D9A002AE0D01E99D5
:10C1200001A802F0DFFB1D98C719216860687A1A20
:10C1300032468241D7D2C91BB0411C9A531A3346AA
:10C14000834100D30A461D92054883691CAA2846EC
:10C15000394698470028DFD0C2E7C04680F9011071
:10C160001CD200305B444247205D2041524D5F5558
:10C1700043505F526561642072657475726E6564C8
:10C1800020302062797465730D0A0000F0B585B027
:10C190000021C943F0B30190009101F085FB0746EF
:10C1A0006F37B7FBF0F141437C1A1C4D2E467036B9
:10C1B000284601F07DFB4519B542F9D33F1B1848CD
:10C1C000874208D218482818874209D9154801F033
:10C1D00091FC30BFFDE7134801F08CFC30BFFDE758
:10C1E0001248FF223946FCF78AFD114802A90A4687
:10C1F00038C838C2019801F0C9FA08B1009909E0BD
:10C2000003987028009905D1084804493A4601F07E
:10C2100057FB01464842484105B0F0BD00A002105E
:10C2200001400000310A02100060FDEFB0D900307B
:10C230008CF90110F0B599B0044600200F900E90D3
:10C240000D900C900B900A90099006900890454F25
:10C25000002A00D180E01E460D4605920CA800F091
:10C2600061FF08B10E3777E00CA8214601F048F9CC
:10C2700020468F30A8426CD804960CAE304601F0B0
:10C280003DF90790304601F035F907994018A8426A
:10C290005FD3281B451C6F08069E07D00026311966
:10C2A0000CA801F02DF98619BE42F8D31E98039010
:10C2B0000996A81B0B90089430190A900820079043
:10C2C0002A4808300290069F0CAC204601F014F971
:10C2D0000646F80008A90D582A46403210A9204603
:10C2E000079B00F037FF78BB069810A9095CB142A4
:10C2F00003D1401C0728F8D926E010A846880398E7
:10C3000000B10660049886421ED80CA805992A46FA
:10C31000334600F01FFFB8B912A8012101758181D1
:10C320001149169100251495E94313910299129130
:10C3300018A96A461160059932462B4600F018FE8E
:10C340001898119988420AD07F1C022FBCD3054F40
:10C35000BF1D0CA800F014FF384619B0F0BD2F46E1
:10C36000F7E7C0460101FF8004010210B805021082
:10C37000F0B5A9B016A848242146FCF7F0FC04AD9E
:10C3800028462146FCF7EBFC2846FFF729FE5249D8
:10C390000B6800249BB14F490A6882B1C0CB059C51
:10C3A0006740049D6E403E43083B16B913785B1C02
:10C3B00002E01D605C600023137009680C7802289D
:10C3C00008D048B9022C09D80598179004981690FF
:10C3D000012709E041A004E0032C01D355A000E0AF
:10C3E00048A001F087FB00275D48426A002504ACA5
:10C3F000284621469047012616A918B1594801F050
:10C4000079FB54E00291344801680029039607D073
:10C4100009C905994B40049A5040184310B902E0ED
:10C420000599049A0120179B169EB21A8B413AD2A5
:10C430003946039A51400843012834D1264608362C
:10C4400003CE0143083E71B3002004A90190FFF719
:10C450001FFEC0B306CE4648081A1046019B9841FD
:10C4600033D220463030029F3B46303310343D46B5
:10C4700010350837059E1796049E169606C7C6CC3B
:10C48000C6C5C6CCC6C536C836C33D4801F032FB6A
:10C49000002616A93046FFF745FDC0B13A4801F025
:10C4A00029FB039E0CE0304801F024FB039E1FB1E2
:10C4B000324801F01FFB03E02F4801F01BFB2E4622
:10C4C000304629B0F0BD2948EEE72A48ECE72D4870
:10C4D000EFE7C046ACD90030381A01305B44424720
:10C4E000205D20416374697665206669726D7761AD
:10C4F000726520736C6F7420697320656D70747938
:10C500000D0A00005B444247205D20416374697658
:10C5100065206669726D7761726520696E74656702
:10C520007269747920636865636B206661696C6504
:10C53000640D0A005B444247205D204661696C65DA
:10C540006420746F20626F6F742061637469766514
:10C55000206170706C69636174696F6E0D0A000010
:10C560001CD200305C0B0210CB0B0210EF0A021041
:10C57000015C0D006E0B02103B0B0210A70B0210AA
:10C58000870B0210CF0A0210150B0210F0B589B00C
:10C5900007460025089507950695059528483860B3
:10C5A00028480860284C386830B10E4605A800F0CD
:10C5B000B9FD18B1093440E0E41C3EE0049605AE34
:10C5C0002249304600F09CFF304600F097FF029071
:10C5D000304600F08FFF019039680391304600F03B
:10C5E0008FFF0399B1FBF0F1414303910498006878
:10C5F0000090411E304600F083FF064638680399DC
:10C60000884217D10098401E2946A94132462B4640
:10C61000FBF778FF0299019A521804990968914230
:10C6200008D8401C4643B14204D105A800F0A8FD3B
:10C630002C4602E005A800F0A3FD204609B0F0BD9D
:10C640000080021000A002100601FF80980E021068
:10C65000B0B50E4800F0C0FD0D480C300021CC43B1
:10C660000325016859B1001D6D1C102DF9D3FBF78E
:10C67000B5FE18210160054800F0AEFD04E004603D
:10C68000024800F0A9FD2C462046B0BD8CD60030F3
:10C6900054D2003082B080B582B00593049220B1AC
:10C6A00004AA01920348FBF7AEFF02B080BC01BCB4
:10C6B00002B00047F0D300302649096801B10847AD
:10C6C0007047C046364800680168084734484068EB
:10C6D0000168084732488068016808473048C068E8
:10C6E000016808472E480069016808472C484069DE
:10C6F000016808472A488069016808472848C069D6
:10C700000168084710B582B0044601F039FA0021EB
:10C710002448234A136873B1121D001D491C0829BF
:10C72000F8D301F06DFA0022684602600748084914
:10C73000134601F037FE1460046801F061FA054801
:10C7400005490160204602B010BDC04620010180AD
:10C75000CE06021028D900305DC7011010B582B096
:10C76000044601F00DFA00210D480E4A1368A34259
:10C770000ED0121D001D491C0829F7D301F040FA04
:10C78000002268460260084808A1134601F00AFE2C
:10C790000021016002B010BC01BC864601F030BA35
:10C7A00008D90030E400021001010180547269656B
:10C7B0006420746F206672656520696E76616C69AD
:10C7C0006420435468756E6B456E74727900000086
:10C7D000F0B581B004464C20205C20B1206D401C97
:10C7E000206500256BE000262665204600F0D8F97C
:10C7F0000546002863D1E068002863D0142145561F
:10C80000E06A08B1E9B206E020461830FFF77AFF87
:10C81000E062E168097DAA002D4B1B689A1810643C
:10C8200048B2002807DB1F21014001228A4040094D
:10C8300080002849425025464C35606940F200117D
:10C84000FEF712FC6069FEF745FC0F21A27C120680
:10C85000120F01D02A7810E0424242411E4803786C
:10C8600047783F02FB188778C0780002C01900049F
:10C87000C01800D0012002402A700F051AB1012013
:10C880002065354605E0207A14A1FFF703FF2A78DA
:10C89000194D207A19A1FFF7FDFE2069384201D019
:10C8A00060680BE00C48417A827A12025118C27A11
:10C8B000007B000280180004401860606060284619
:10C8C00001B0F0BD11481249E12201F0D3FCC0468D
:10C8D00008ED00E000E100E05CD400304661696CE6
:10C8E00020746F20696E697469616C697A65206370
:10C8F0006172640A000000005FF0FFFF696E6974F6
:10C900002063617264203D2025640A00080602103D
:10C910001D060210F0B587B00D4606460068C16BD3
:10C920000D9C684644600C9F076030460592069354
:10C93000884701467C4839B34C210396715C002935
:10C94000069B56D0794801218907491BB9421DD35E
:10C9500003210F2212072A401E460B079A42334634
:10C9600014D129403A4602400A437AB90598400A50
:10C97000D9054218780AE105431803984069294609
:10C98000FEF7F0FB90BB34E0401C32E03946214317
:10C9900071B3411C0291059A0592500A0693D9057C
:10C9A0004218780AE10540180494610A01430029FD
:10C9B000029E00D13E46730A039840695C4C2146B2
:10C9C000FEF7D0FB90B9284621463246FCF748F9DD
:10C9D0000020BF1B049C844139462143059A9219CB
:10C9E000069B4341AD190029D6D102E0D54800E0AD
:10C9F000002007B0F0BDC046017270474C21405C7A
:10CA000008B10020704748487047C046B0B504469A
:10CA10004C20205C20B1206D022803D3401E0AE088
:10CA2000002008E025464C35E06810B1406802F06F
:10CA30003FFE0020287020650020B0BDF0B587B013
:10CA40001446059107460068016C0D9E68464660D5
:10CA50000C9D05603846069388470146324851B31D
:10CA60004C210397795C0029059F5AD033462F4902
:10CA700001229207D21BAA4228461ED303250F2269
:10CA800012073A401E462B079A423346274914D1D3
:10CA90003D4002460A402A437AB9610A069AD20505
:10CAA0008A18400ADB05C318039840693946FEF727
:10CAB00081FE98BB35E0401C33E002461A437AB34E
:10CAC000491C02910146480ADA05801805935A0A62
:10CAD0000243002A029D00D10D46049114483946B4
:10CAE0002A46FCF7BDF8600A2646069CE105421876
:10CAF0006B0A039840690E49FEF75CFE70B900208E
:10CB00000499491B059B83410A461A4376194441FF
:10CB100006947F19002A3446D5D102E0894800E006
:10CB2000002007B0F0BDC04674ECFFFFFF0100001D
:10CB300008D70030416917480A58D20707D00818AB
:10CB40000122026040F600000B5813430B50124ABA
:10CB500088188958C90703D0104901220A70026059
:10CB60000168C90502D540F200110160016889071A
:10CB700001D5022101600168890402D542F2000159
:10CB800001600168C90404D541F2000102680A434A
:10CB900002607047080800002C080000351A0130B8
:10CBA000F0B581B00446007A49A1FFF773FD206B10
:10CBB000514901F097FF0090606B504901F092FFDE
:10CBC0000646A06B4E4901F08DFF0746E06B4D49CC
:10CBD00001F088FF05460098314601F063FF0646E4
:10CBE0003846294601F05EFF0146304601F05AFF03
:10CBF0000090206C444901F075FF0646606C434983
:10CC000001F070FF0746A06C414901F06BFF05463B
:10CC10003046394601F046FF294601F043FF014600
:10CC2000009801F03FFF0546401C3CD0394928469A
:10CC300001F002F8E060F0B30068A84241D1206B37
:10CC40002D4901F081FF606B2C4901F07DFFA06B45
:10CC50002B4901F079FFE06B2A4901F075FF206C48
:10CC6000294901F071FF606C284901F06DFFA06C4B
:10CC7000274901F069FF31482E46064002F01EFDAB
:10CC800025616661E068006902F01EFDE268121D20
:10CC900007CA02F01FFDE068406802F021FD02F0C3
:10CCA00025FD002005E02068C26C01212046904748
:10CCB000244801B0F0BD22481F4940F2DF1201F0C4
:10CCC000D9FA40F2DF10421C13A01B4901F0D2FA3E
:10CCD0005344204D50462053657474696E67202676
:10CCE00020456E61626C6520534420495020436C9E
:10CCF0006F636B0A00000000F8FA01101CFB0110C2
:10CD000040FB011064FB0110D4FA0110B0FA0110CD
:10CD100098FA0110AC0002105F7364685F6D6F6475
:10CD2000696E69742D3E6D6F646E616D65203D3D69
:10CD30002073645F6D6F64001D060210E0FF0FFF3B
:10CD4000080602105FF0FFFFF0B581B04C22002111
:10CD500081548162124A426201624161C160017282
:10CD60004160016540F200120E4B8361CB430361C9
:10CD70001B4B0833036040F200130C33541C009427
:10CD8000551D161DD71C941CC1620463476386633E
:10CD9000C5630264009941648364C06101B0F0BD61
:10CDA00035CB0110B1D1011080B500F005F880BC81
:10CDB00002BC8E4600F0A8BB10B5044608480830F7
:10CDC00020604C20205C10B12046FFF71FFEE06A77
:10CDD00018B1FFF771FC0020E062204610BDC0468C
:10CDE0000405021000200870012070471D207047C4
:10CDF0001520C0437047002070471046704701203F
:10CE00007047FBF720BB1520C043704711B91820AD
:10CE1000C0437047002070471520C0437047016829
:10CE2000896A08470020704701680B6900210122C8
:10CE3000184701688969084703681B6918477047E4
:10CE400001680B6900210A4618471520C043704746
:10CE50007047000010B50C48D0E88F0FC00701D014
:10CE60000A4810BD084800F077FB0028F8D0074CAE
:10CE70002046FFF769FF0648064A214600F06AFB94
:10CE8000014800F093FBEBE784D6003044D9003032
:10CE9000B9CD0110008001100020704700207047BC
:10CEA00070B50F2801DD002419E005468000114906
:10CEB0000C58022D13DC621C11D10E18284600F00C
:10CEC0001FF8044650B9284600F01CF8044628B95B
:10CED0000948D0E88F0FC007084C02D034602046C4
:10CEE00070BD054800F038FB0028F7D0024800F07C
:10CEF0005DFBF3E754D2003080D6003094D200308E
:10CF0000002070470020704790B4047D022C04D0AC
:10CF1000012C05D190BC00F05FBA90BC00F09CBA27
:10CF20000020C04390BC704770B5C1B10A68437B14
:10CF300063B100232024D50703D0651E0126AE402F
:10CF40003343641E5208002CF5D100E0134682687A
:10CF50005A400A60016889688847002070BD1748F8
:10CF6000174940F2131201F085F9C04670470000DE
:10CF700070B582B0069CDCB105464068206068460A
:10CF800004602846FFF7C0FF28B10646286881687C
:10CF90002846884709E028462146FFF7C5FF18B113
:10CFA00006460020206000E00026304602B070BD3A
:10CFB00002480349A12201F05DF9C0465206021061
:10CFC0005E06021000F0A0BA7047007B70470000B8
:10CFD000F0B581B00E460446174800F0FDF817483A
:10CFE00005680DE0AF6857B13846FBF717FEB04251
:10CFF00005D1384621463246FBF7E2FD88B16D681F
:10D00000002DEFD1072E05D10DA007222146FBF7F9
:10D01000D7FD50B1084800F0DFF80025284601B0E0
:10D02000F0BD054800F0D8F8F8E7034800F0D4F860
:10D0300005480568F2E7C04630D900302CD90030E9
:10D0400064656661756C740038D90030B0B505460A
:10D050004068002430B1FFF7B8FF012802D16C68A6
:10D0600004B1241F2046B0BDB0B505464068002479
:10D0700028B1FFF7AAFF10B96C6804B1241F20463D
:10D08000B0BD406800B10120704780B5406828B14C
:10D09000FFF79BFF01464042484180BD002080BD14
:10D0A0000068704770B50E4604460025056045606F
:10D0B0000EA13046FBF774FD301802E02F2A06D08F
:10D0C0006D1C41192160425D002AF7D101E0491C25
:10D0D00021602DB12946FFF77BFF6060204670BDBF
:10D0E00003A006A12A2201F0C5F8C0462F000000C7
:10D0F0006C656E20213D2030000000002E5C6D62CA
:10D1000065642D6F735C706C6174666F726D5C73B7
:10D110006F757263655C46696C65506174682E63F7
:10D120007070000070B50546204E304600F054F88F
:10D13000284602F0E1FA0446284602F0E3FA00F03D
:10D14000E5F9E860304600F047F80CB10020C44330
:10D15000204670BDF0B581B01C4615460E46074608
:10D16000124800F039F8384629463246234600F086
:10D170005CFD04460D4800F02FF8204601B0F0BDDC
:10D18000B0B50546094800F027F8284602F0C0FA75
:10D1900008B9044601E00020C443E86808B100F083
:10D1A000B1F9024800F018F82046B0BD3CD9003073
:10D1B00030B4436873B1C268056901242C4021462C
:10D1C000114339B18168681018180CB103689A5876
:10D1D00030BC104730BC704780B50146006808B9C4
:10D1E000086818B1091D884203D180BD081D086078
:10D1F00080BD02A00AA18B2201F03CF870203D3DC9
:10D20000207265696E746572707265745F636173B4
:10D21000743C54202A3E28265F6461746129000012
:10D220002E2F6D6265642D6F735C706C6174666F18
:10D23000726D2F53696E676C65746F6E5074722EC9
:10D2400068000000002140F200207047002140F2F9
:10D2500000207047002140F200207047002140F27A
:10D26000002070474C21425C002112B1406840020E
:10D270007047C9430048704774ECFFFF00A0704737
:10D280004E555344000000000120704711207047A4
:10D29000F0B585B01D46164604460068416A204632
:10D2A000884702460B4630462946FBF72BF91343C5
:10D2B00000270BBB019603950B9D0A9E2068416ACF
:10D2C0002046884702460B4602963046049529467A
:10D2D000FBF718F913437BB9029801994618049D8E
:10D2E000039845412068816B20468847801BA941EF
:10D2F00001D2002700E00127384605B0F0BDF0B5A7
:10D3000081B01C46164605460068016B28468847D2
:10D3100002460B4630462146FBF7F4F813430BB1A7
:10D3200000261BE0079806998F19444100267A1EB3
:10D330002346B3412868016B2846884702460B46BE
:10D3400038462146FBF7DEF813433BB92868816B6A
:10D3500028468847C01BA141E2D30126304601B0D0
:10D36000F0BD0020C0437047F0B585B01D4616469D
:10D3700004460068816A2046884702460B463046CC
:10D380002946FBF7BFF8134300270BBB0196039513
:10D390000B9D0A9E2068816A2046884702460B46FC
:10D3A0000296304604952946FBF7ACF813437BB947
:10D3B000029801994618049D039845412068816BA5
:10D3C00020468847801BA94101D2002700E00127A1
:10D3D000384605B0F0BD0000F0B587B006910C9C52
:10D3E000A4B3114619430194256851B3016903910F
:10D3F000007B029000273C46059304920698C65D88
:10D40000029860B100210823F20703D05A1E0120C0
:10D41000904001435B1E7608002BF5D100E03146B9
:10D4200000207F1C4441280EC9B241408800039966
:10D4300008582D024540049AB81A2046059B984189
:10D44000DCD301980560002007B0F0BD27482849CB
:10D4500040F2D91200F00EFFF0B587B005910C999B
:10D46000D9B314461C430191096884B30691039211
:10D47000007B029000251C4E2F4604930598445DC6
:10D48000029860B100200823E20703D05A1E012150
:10D49000914008435B1E6408002BF5D100E0204654
:10D4A0000406069844400820049B6100002C00DA22
:10D4B00071400C46401E0106F7D100206D1C47410B
:10D4C0000398281A384698410694D7D300E00C46B2
:10D4D00001980460002007B0F0BD0448044940F200
:10D4E000AD1200F0C7FEC046B71DC10452060210BF
:10D4F0005E06021002F012B902F016B902F01AB973
:10D5000002F01EB9FAF79FBFFAF79DBF10B582B0BF
:10D510000446FAF767FF08B102B010BD0023684661
:10D520000360024802A1224600F03CFF1F01018077
:10D530004F70657261746F72206E65775B5D206FEE
:10D540007574206F66206D656D6F72790D0A00002D
:10D550007046F0470120704780B5014603780322EA
:10D5600013400020012B04D00B781A4012B1012A7D
:10D5700005D180BD022003430B70012080BD02A0B5
:10D580001349094A00F076FE286775617264202607
:10D59000204358415F47554152445F4D41534B2909
:10D5A000203D3D20300000009D06000080B5017840
:10D5B00003220A40022A04D1FC221140491C0170B6
:10D5C00080BD02480249034A00F054FE1D080210C3
:10D5D00054080210A606000090B406480168842290
:10D5E000054B10C910C3521EFBD10349016090BC0A
:10D5F00000F054BF08ED00E000D0003000F09EBA0B
:10D60000FEE710B5FFF74CFC28B10168896A88472E
:10D61000002802DB10BD092400E04442FAF7DEFED8
:10D6200004600020C04310BD00F084BDB0B50D46BD
:10D6300004462149FBF796FBB8B120492046FBF789
:10D6400091FBA0B11E492046FBF78CFB88B12078E6
:10D65000402814D16078A17809020818E17822796D
:10D660001202511809040C1807E0002402E00124FA
:10D6700000E002242046FFF713FC2046B0BDA807B7
:10D6800006D4680706D42807C1170920084002E01D
:10D69000022000E001202907890F02D040F200217A
:10D6A0004018290240F200420A4081182046B0BCCE
:10D6B00004BC964601F06CB9D4050210DB050210DB
:10D6C000CC050210002200F047BD10B5002A07DB90
:10D6D000144662B1224601F0A4FF002808DA03E0F4
:10D6E000FAF77CFE162101600020C04310BD002027
:10D6F000201A10BD80B582B001A908700120024631
:10D7000001F08FFF02B080BD80B51248006801684B
:10D71000C96A884780BDC04680B50E480068016868
:10D72000896A884780BDC0460A48006801688968E0
:10D730000847C04670B582B00146064800680468D4
:10D74000646900256E467560069D3560A04702B08D
:10D7500070BDC0469CD9003070B599B10022D44349
:10D760000822094B05786C40491E15466608E407F7
:10D7700000D05E4034466D1EF8D1401C0029F1D126
:10D78000E04370BD002070BD2083B8ED70B5064643
:10D790000220BEB30C46A9B32168702932D3A06819
:10D7A00070252946FBF7D9FAA068174900F088F9D7
:10D7B000A068001D022100F083F90CCEA06808309B
:10D7C000083E00F086F9B268F368A068103000F0F7
:10D7D00080F9A0683146103118302022FBF740FA5A
:10D7E000A0683036583010223146FBF739FAA0686D
:10D7F0006C21FFF7B1FF0146A0686C3000F060F9C2
:10D800006560002070BDC046D4B3515AF0B581B0F8
:10D810000E4605464D4F384601F08CFF044638460B
:10D8200001F07CFF0019A84211D9AC420ED2474F3B
:10D830003846214601F084FF0419AC42F8D30EB9F2
:10D84000204600E0201AAC4200D00446204601B039
:10D85000F0BDC046F0B581B00D4604460121FFF78A
:10D86000D5FF0746281900252946FFF7CFFFA74215
:10D8700012D10646A04210D9344F3846214601F055
:10D8800065FF05463846214601F05AFF0419B442A7
:10D8900003D2002DF1D000E0ED43284601B0F0BDE9
:10D8A0002A4801F035BFC046284801F02BBFC046CA
:10D8B0000146264801F044BF244801F01DBFC04680
:10D8C000F0B583B00025EF43019010B300921F4ED6
:10D8D0003046029101F02EFF0446304601F01EFF53
:10D8E00002998C4215D8009EB04212D300197118CB
:10D8F00081420ED8154801F005FF02990446B1FB9C
:10D90000F0F06043081A04D1B6FBF4F06043301A1B
:10D9100002D0384603B0F0BD002E2F46F9D00025C6
:10D920004919019842190948234601F015FF074695
:10D930000028EED12D19B5420299F1D3E9E7C0468E
:10D9400013460246014800F070B9C046A0D9003025
:10D95000F0B59BB0022600284DD00C4600294AD0D5
:10D96000054613AE202730463946FBF7F8F91296E4
:10D9700000261196109710A8FDF708F908B10226A5
:10D9800039E001960F95E8200E900D9005AE3046D7
:10D990003946FBF7E4F904960397029710A80DA9FE
:10D9A00002AAFDF75DF8022628BB0E970D972846C0
:10D9B000E8300F900DA802A9FCF77AFFD8B92846E5
:10D9C000083000F058F803C428461030083C00F036
:10D9D00052F8A060E160204610302946183120221C
:10D9E000FBF73EF920463030A03510222946FBF7E0
:10D9F00037F9019E266430461BB0F0BDF0B581B00A
:10DA0000022638B30D4629B304466C21FFF7A4FE65
:10DA1000074620466C3000F020F8B8421AD1204664
:10DA2000083000F028F803C520461030083D00F00B
:10DA300022F8A860E96028461030214618312022DB
:10DA4000FBF70EF930355834102228462146FBF7F3
:10DA500007F90026304601B0F0BD50B14178027898
:10DA6000120251180902827889180902C078081830
:10DA700070470020704700B34178027812025118B5
:10DA80000902827889180902C27889180A0E1202DE
:10DA900009020379C9180B0ED21812020902437940
:10DAA000C9180B0ED218120209028379CB18190E6D
:10DAB00051181A02C07910187047002001467047AB
:10DAC00030B1C1700A0A82700A0C4270090E0170EE
:10DAD000704768B1C271110A8171110C4171110E48
:10DAE0000171C370190A8170190C4170190E01700F
:10DAF00070470000B0B504460E48017861B90121B5
:10DB000001700D4D07210622284601F041FAE1205F
:10DB10004102284601F0C6F9217849B1651C064C3E
:10DB2000204601F0E9FA681C297800290546F7D15A
:10DB3000B0BDC04688D6003094D6003010B504463B
:10DB4000FFF7AEF9A100094A0024545030B1016832
:10DB500049698847002807DA444200E00924FAF7B7
:10DB60003DFC04600020C443204610BD54D2003068
:10DB70000120EFF310810140484248417047000006
:10DB800080B500F09FF905480168491C01D001608B
:10DB900080BD03A00FA13F2200F06CFBB41901303F
:10DBA000637269746963616C5F73656374696F6ED6
:10DBB0005F7265656E7472616E63795F636F756EB7
:10DBC000746572203C2055494E5433325F4D4158A4
:10DBD000000000002E5C6D6265642D6F735C706CDC
:10DBE0006174666F726D5C736F757263655C6D6294
:10DBF00065645F637269746963616C2E6300000021
:10DC00000448016811B1491E016000D0704700F05E
:10DC100067B9C046B4190130EFF3058000B10120A7
:10DC2000704700B9FEE700F053FB80B510461A4676
:10DC3000FBF716F8002080BD10B561B102460B68F5
:10DC4000002003E0934204D0CB691C315C1CF9D165
:10DC500010BD084610BD02A006A1172200F00AFB65
:10DC60006D6F6470726F705F74616220213D204E31
:10DC7000554C4C002E5C6D6265642D6F735C746155
:10DC800072676574735C5441524745545F4E5556F4
:10DC90004F544F4E5C6E755F6D6F647574696C2E7A
:10DCA0006300000000487047A80C0210F0B581B076
:10DCB0000A4604460068411C21D02272617A062976
:10DCC00055D8860840F2C0331E407B4D731900932F
:10DCD000C3B28F0001A5ED19AF46C04600F011B8E0
:10DCE00000F01CB800F027B800F006B800F004B847
:10DCF00000F03DB800F02DB8BAB3042136E001B011
:10DD0000F0BD01261F469E400022009D2846314658
:10DD1000FCF77DFF607A012804D009E001261F4648
:10DD20009E40009D022228463146FCF770FF607A33
:10DD300002283B4605D10122114699400098FCF784
:10DD400066FF207A08B1042100E003216172206897
:10DD50000DE006215AB95A4AB21840F2C0333C339A
:10DD600084001C400123135101E00321617201B0C2
:10DD7000F0BC04BC964600F051BEC046B0B50446A7
:10DD80000160481C0BD00D460021284600F044FEDF
:10DD900040F200202081E8B2012181406160B0BDE5
:10DDA000002200F001B8000070B515460E4604468A
:10DDB000FFF7E4FF701C1DD02068411C1BD001211F
:10DDC000002D0A4600D12A4640F2C03340F2C03549
:10DDD0003C3586002E4080081840394BC0188251CF
:10DDE0002046FFF763FF0021204670BC04BC964626
:10DDF00000F00AB870BD024802492A2200F03AFA3F
:10DE00007A06021092060210F0B581B0044600684E
:10DE1000421C22D0062938D8850840F2C03215406D
:10DE2000254BEB180093C6B28F0001A3DB199F4668
:10DE300000F015B800F017B800F019B800F006B8F7
:10DE400000F004B800F021B800F021B803292AD16D
:10DE500040F200312181032128E001B0F0BD012111
:10DE6000B140002206E00121B140022202E001227D
:10DE70001146B1400098FCF7CAFE207A08B104218F
:10DE800000E003216172206810E061720EE006215B
:10DE90006172237A53B90A4BEB183C328400144068
:10DEA00001221A5102E005492181042101B0F0BC90
:10DEB00004BC964600F0B2BD0040005001040000D2
:10DEC00000480050EFF31080EFF3108172B60D4957
:10DED0000A7822B901220A7082430B480270704707
:10DEE00080B5EFF31080C00707D00648002101700D
:10DEF0000548007800B162B680BD04A00AA13622B0
:10DF000000F0B8F9841A0130B0190130216172654E
:10DF10005F696E74657272757074735F656E61624D
:10DF20006C656428290000002E5C6D6265642D6FAD
:10DF3000735C68616C5C6D6265645F63726974696F
:10DF400063616C5F73656374696F6E5F6170692E86
:10DF50006300000070B58EB014460D46064601A859
:10DF6000001D3021FAF7FBFE0395002E00DB184E52
:10DF7000019618483018032802D8686BEC6B00E053
:10DF800001A808900294FFF7FBFD134801684A1CA2
:10DF9000026049B901A811491CC81CC11CC81CC198
:10DFA0001CC81CC13CC83CC101A80D491CC81CC1EF
:10DFB0001CC81CC11CC81CC13CC83CC10948016824
:10DFC00009B107488847FFF71BFE0EB070BDC04679
:10DFD0000101FF80C3FE007FB8190130001A013033
:10DFE0003C1A0130BC190130F0B587B004464068D6
:10DFF0003821415C11B93A21405C08B107B0F0BD4D
:10E0000005912068006880472068C06980470568DE
:10E01000002D4DD01F2601270021F2B23B46934030
:10E020009D4203D0761E3206F7D10E460697406811
:10E030000490001F02901D2843D2606800270760EB
:10E040004760206840688047039464683B216654B9
:10E05000059967542062A560A762E762276367633A
:10E060000726029886401B4A304639463B46FAF757
:10E0700031FA28187941401EB9412A463B46FAF741
:10E0800041FAA061E1612661F8430146049AFAF77A
:10E0900000FAC043E06006982087039C204601F008
:10E0A00049F9204607B0F0BC02BC8E4600F064BEC1
:10E0B0000022684602600848093017A1134600F0A4
:10E0C00071F9002268460260034804A1134600F07B
:10E0D00069F9C04640420F00050104805469636B32
:10E0E0006572206E756D626572206F66206269745C
:10E0F0002069732067726561746572207468616E4F
:10E10000203332206F72206C657373207468616EE7
:10E1100020342062697473005469636B65722066F1
:10E1200072657175656E6379206973207A65726FA7
:10E130000000000010B5FEF7B3FE28B10168C96900
:10E140008847002802DB10BD092400E04442FAF7AA
:10E1500045F90460002010BDB0B514460D46FEF729
:10E160009FFE38B101680B6929462246984700286E
:10E1700002DBB0BD092400E04442FAF72FF9046045
:10E180000020C043B0BD000010B51748006C082047
:10E19000FAF728F9154908600120FAF723F9144C19
:10E1A000206014A0FFF7A6FC17480068804708B15C
:10E1B00016A014E0FDF7C0FD80B1FEF7D9F838B124
:10E1C000FDF7C0FD25A0FFF795FC284800F070F989
:10E1D000206808B100210170254800E015A0FFF774
:10E1E00089FC0020C04310BD68000210381A0130BD
:10E1F000ACD900300D0A4D62656420426F6F746CBB
:10E200006F616465720D0A001CD200304661696C52
:10E21000656420746F20696E697469616C697A65E0
:10E22000207570646174652073746F726167650D29
:10E230000A0000004661696C656420746F20696E95
:10E24000697469616C697A652061637469766520B7
:10E2500073746F726167650D0A000000626F6F74FE
:10E26000696E672E2E2E0D0A0D0A000000A4021002
:10E27000AE0A021082B00B460146684602600248B0
:10E28000002200F08FF8C0464401FF80B0B584B092
:10E2900004460025039502950195FF20A4B110299D
:10E2A00012D303A802A9FEF771F901060CD1029955
:10E2B000039801AA6B461A6010232246FDF7BAFFA5
:10E2C0000199102900D0E84340B204B0B0BD00006D
:10E2D00086B0FFF755FC40F2C031BE3903A8FFF706
:10E2E0005FFD002540F2C0303C30029001200190DB
:10E2F000009545E08100029F3940800840F2C0321D
:10E300001040254E3043019A4250214C204601F0E6
:10E3100079F90398411C36D081003940800840F2D9
:10E32000C03210403043009A4250204601F06AF952
:10E330006D1C042D24D3009C0398411C23D0810024
:10E34000029D2940800840F2C0321040124F3843ED
:10E35000019A42500F4E304601F054F90398411C87
:10E3600011D081002940800840F2C032104038436B
:10E3700000254550304601F045F9641C042CDBD3E0
:10E380000398411CB6D1054805492A22FFF772FFC0
:10E39000F0490200801A0600004800507A06021078
:10E3A0009206021082B001930D460121094BD3E879
:10E3B0004F7FC3E8441F39060AD17646029F1146B3
:10E3C0007246FFF7C7FD284601993A4600F0EEFB7A
:10E3D00000F044F8701A013083B080B581B003AF0B
:10E3E0000EC703A9009100F01DF801B080BC01BC6C
:10E3F00003B00047B0B50446022500222846214656
:10E4000001F00FF9FFF7BCFB2046FAF707FC0246C4
:10E410002846214601F005F9B0BC01BC8646FFF74D
:10E42000EFBB000010B5A2B00B46024601A8842144
:10E43000FAF7F0F80446842805D301A87F3005A137
:10E440000522FAF70DFC012C02DB01A8FFF7D2FF31
:10E4500022B010BD2E2E2E0A0000000001200D4A11
:10E46000D2E84F1FC2E8430F002BF9D1C80705D0EF
:10E47000FFF786FBBFF34F8F20BFFDE7FFF7CCFB15
:10E4800028B9FFF775FB10B10120FFF7CAFBFFF7B2
:10E490001FFFC046361A013070470000034801785C
:10E4A00001B1704701210170FDF754BA741A0130AF
:10E4B000F0B5EFF3108172B6174A00211160CA431C
:10E4C000164B174C174D0E46B7003A517A510F466E
:10E4D000D9513F1D202FFBD12033761C082EF3D1BC
:10E4E00005214A0610490A604860104A8A600022E5
:10E4F000CA601346CC18A2611B1D082BFAD100225A
:10E500000A6201684068002282F314888D4682F313
:10E5100010880047F0BDC04610E000E000E400E0D5
:10E5200080E100E080E200E004ED00E0FA05000098
:10E53000F0B5D7B00191009008300FA93CC83CC19C
:10E540003CC83CC13F20C04305900024129808906D
:10E5500011980690109D0F980A90149F15980E9090
:10E560001398099016980790099E0E9A0A9B06998F
:10E570000F2C0E9704940D960C9503920B9110D8C6
:10E580000198059A80184021415C09064125455DA6
:10E590002D0469184225455D2D0249194325405D2A
:10E5A00018E017A8059A81588018456A4919856BA3
:10E5B00013262F46F741AE0A7E401127FD417540D4
:10E5C0004919406812250646EE41C50875400726E0
:10E5D000F0416840091817A8801801640C9D28466E
:10E5E00018401D430B9E354005430B200D9C2646CD
:10E5F0000293C64106202746C74177401920264688
:10E60000C6417E4025488018006C079BC0188019C1
:10E610004618029B0E9903984140214041407418CE
:10E6200029190D251E46EE4102251F46EF41774070
:10E6300016251E46EE417E4089190A91089909194E
:10E640000991121D049C641C0592C02A0D9A0B9915
:10E650000E4608910C9D294606951D4617460790C3
:10E6600082D10E9C1594099C1394169014921296C4
:10E67000119110930A990F91009CA0684018A06016
:10E680000FA8001D0C340021425863589A1862509C
:10E69000091D1C29F8D1002057B0F0BD98F90110D0
:10E6A00021B10A4602490B68002118477047C0464D
:10E6B00004060210C046C046F0B581B00C460546BF
:10E6C00007683F223946114006462836802070549C
:10E6D0004B1CF018382B04D83722511AFAF73DFB9F
:10E6E0000BE05140FAF739FB28463146FFF720FF8F
:10E6F00038213046FAF733FB2F68F8006721685459
:10E70000780966216854780B65216854780D642176
:10E710006854686841096222A954410B6122A954D6
:10E72000410D6022A954790FC0004018632168543C
:10E7300028463146FFF7FCFEE87A20706889607051
:10E74000A868000AA070A868E070E87B2071E889DA
:10E750006071E868000AA071E868E071E87C2072E6
:10E76000688A60722869000AA0722869E072E87DF0
:10E770002073E88A60736869000AA0736869E073AF
:10E78000E87E2074688B6074A869000AA074A86988
:10E79000E074E87F2075E88B6075E869000AA07571
:10E7A000E869E0752320285C2076688C6076286A0A
:10E7B000000AA076286AE076A86E48B92720285C6F
:10E7C0002077E88C6077686A000AA077686AE0774B
:10E7D000002001B0F0BD10B16C21FFF761BF7047A0
:10E7E00080B56C21FAF7BBFA80BD0000816600227B
:10E7F0000260426009B12C4A00E02A4A426209B133
:10E800002B4A00E0294A026209B12B4A00E0294A5A
:10E81000C26109B12A4A00E0284A826109B12A4A44
:10E8200000E0284A426109B1294A00E0274A026112
:10E8300009B1294A00E0274AC26009B1284900E02D
:10E84000264981607047C0468166002202604260AE
:10E8500009B1154B00E0134B436209B1144B00E0C2
:10E86000124B036209B1144B00E0124BC36109B1B2
:10E87000134B00E0114B836109B1134B00E0114BC6
:10E88000436109B1124B00E0104B036109B1124B17
:10E8900000E0104BC36009B1114900E00F498160ED
:10E8A0001046704719CDE05BA44FFABEABD9831F69
:10E8B000A78FF9648C68059B111558687F520E511B
:10E8C000310BC0FF3AF54FA539590EF772F36E3C84
:10E8D00017DD703085AE67BB07D57C3667E6096A01
:10E8E000D89E05C1C046C046F0B583B0E2B3144619
:10E8F0000D46064601688A1802603F2308460193C8
:10E9000018408A4202D27168491C71600022A8B185
:10E9100040210F1AA74201D902460FE031462831A3
:10E9200000910818294602923A46FAF799F93046BA
:10E930000099FFF7FDFD029AE41BED19402C0CD362
:10E940000292274630462946FFF7F2FD403F403508
:10E950003F2FF7D801980440029A2CB1B018283004
:10E9600029462246FAF77CF9002003B0F0BD0000EA
:10E9700006480021017000F06BBDC04680B500F074
:10E980007BFD02480121017080BDC04698D900304E
:10E99000F0B585B00D460646FDF75AFE0446002840
:10E9A00035DB0027049702A83146FEF77BFBFEF714
:10E9B00068FBF8B102A8FEF768FB20B102A8FEF7D9
:10E9C00053FB049020E002A8FEF740FB90B10646FE
:10E9D00002A8FEF765FB024630688068019004A932
:10E9E00030462B46019DA84768B14542F9F7F6FC31
:10E9F000056003E0F9F7F2FC13210160A00005496E
:10EA00000F50FC4303E00498A100024A50502046F6
:10EA100005B0F0BD54D2003000F0A4BE80B5421C59
:10EA200012D0C91ECAB2032A0DD8C3B2012199401F
:10EA3000800840F2C03303400648181880BC08BC68
:10EA40009E46FCF7CAB880BD03A008A12922FFF7A3
:10EA500011FCC0460040005070696E20213D202806
:10EA600050696E4E616D65294E4300002E5C6D62EB
:10EA700065642D6F735C746172676574735C544177
:10EA8000524745545F4E55564F544F4E5C54415279
:10EA90004745545F4D323335345C70696E6D61703B
:10EAA0002E63000080B582B0024688420BD0501C15
:10EAB00008D0481C07D0002368460360034804A11F
:10EAC000FFF770FC0A46104602B080BD300101809D
:10EAD00070696E6D6170206D69732D6D617463680E
:10EAE0000000000010B582B002460120C043531C54
:10EAF00015D00B685C1C06D00C3193420AD00B6811
:10EB00000C315C1CF9D1002368460360054806A15E
:10EB1000FFF748FC80000858411C01D1F3E7401C76
:10EB200002B010BD3001018070696E6D6170206EA1
:10EB30006F7420666F756E6420666F7220706572E8
:10EB40006970686572616C0010B582B00446401C43
:10EB50001DD00868421C06D00831A0420BD048687E
:10EB60000C31421CF9D100236846036009480AA110
:10EB70002246FFF717FC09682046FFF74DFF0021EA
:10EB8000204602B010BC04BC9646FFF747BF02B057
:10EB900010BDC04630010180636F756C64206E6FDC
:10EBA000742070696E6F757400000000F0B581B05C
:10EBB00000920D460646032040073E4C21680A4657
:10EBC0000240824201D08FB200E04F42080CC3B233
:10EBD00039483A46FFF700FC38483818132844D81B
:10EBE000810001A251188F4600F026B800F027B826
:10EBF00000F028B800F029B800F02AB800F02BB8CF
:10EC000000F02CB800F02DB800F02FB800F02DB8AF
:10EC100000F02BB800F029B800F027B800F025B8B4
:10EC200000F023B800F021B800F01FB800F01DB8C4
:10EC300000F01BB800F03AB8A168474813E0A1689B
:10EC400041A010E0A1683CA00DE0A16835A00AE059
:10EC5000A1682FA007E0A16824A004E0A16827A074
:10EC600001E0A1681BA0FFF7B7FB3046FFF7C2FB2E
:10EC700061683A48FFF7B0FB4DB139A0FFF7BAFB26
:10EC80002846FFF7B7FB38A00099FFF7A5FBA1685E
:10EC90003648FFF7A1FB21683548FFF79DFB354853
:10ECA00001B0F0BC02BC8E46FFF796BB04A0FFF794
:10ECB00093FBDAE73C1A013057070210CFFEFFFF43
:10ECC000417373657274696F6E206661696C656407
:10ECD0003A2000004D657373616765517565756510
:10ECE0003A20307825582C200000000054696D65CA
:10ECF000723A20307825582C200000004576656E49
:10ED000074466C6167733A20307825582C200000D7
:10ED10004D656D6F7279506F6F6C3A203078255861
:10ED20002C20000053656D6170686F72653A203069
:10ED30007825582C200000004D757465783A2030F5
:10ED40007825582C200000005468726561643A20D0
:10ED5000307825582C200000420702100D080210C0
:10ED60000A46696C653A20002B256400FA070210F8
:10ED7000A807021028070210F0B581B004464668C3
:10ED80003A20305C10B93920305C08B101B0F0BDD8
:10ED9000204600F0CFFA67687968E1B103C93B6BA0
:10EDA0007A6B1D1A15468D4148D2C01A91413D69B2
:10EDB000BA69FB69121A8B4128D3BA68264B9A426A
:10EDC00021D03B23FB5C93B11A46F9F762FB002389
:10EDD000224A801813E0306AF1683269101808403E
:10EDE0002168096901B0F0BC04BC964608470023BD
:10EDF0000093009BF9F76EFB184A8018009B59415D
:10EE0000154AF9F77FFB854200D30546386A401959
:10EE1000FD680540306A854217D0206801692846A0
:10EE20008847206840688047316A8D4202D9A842ED
:10EE300002D303E0A842A9D38842A7D22068406940
:10EE400001B0F0BC02BC8E46004705A00DA140F207
:10EE50001B12FFF70FFAC04640420F003F420F005F
:10EE60006D617463685F7469636B20213D20717507
:10EE70006575652D3E7469636B5F6C6173745F7259
:10EE8000656164002E5C6D6265642D6F735C686102
:10EE90006C5C6D6265645F7469636B65725F617001
:10EEA000692E630003689C4A1A409369DB00FCD515
:10EEB00041611046FCF700BEB0B582B0044605685B
:10EEC000254828408569ED00FCD54D1F042D2ED224
:10EED000052A32D25D1E022D36D218340EC4052901
:10EEE00003D0062903D1012406E0002404E0072909
:10EEF00001D0032400E002240221114303290DD193
:10EF00000825991E4A424A4191006A461160002133
:10EF100022462B46FCF756FE02B0B0BD1825042A47
:10EF2000294600D00021022AEBD00D46E9E70B4824
:10EF30000B4940F26212FFF79DF940F26210421C49
:10EF400008480749FFF796F940F26210821C06A0B4
:10EF50000349FFF78FF9C046E0FF0FFF04090210D5
:10EF600070090210800802102873746F705F626964
:10EF70007473203D3D203129207C7C202873746FE0
:10EF8000705F62697473203D3D20322900000000EB
:10EF9000F0B583B017460D460446FFF77FFA4249A5
:10EFA0002846FFF79FFD064640493846FFF79AFD81
:10EFB00001463046FFF776FD2060411C5ED000958B
:10EFC0003B49FEF739FE00285DD022680168914276
:10EFD0005ED13D460290806901900027FE43009873
:10EFE000211D61C126613049FFF7AEFD2F4928463A
:10EFF000FFF7AAFD019B1868E8B9029D2A1D07CA00
:10F0000000F068FB686800F06BFB286900F05CFBAF
:10F0100021682A4808408169C900FCD5E1214902DC
:10F020006161FCF749FD0821002201232046FFF71A
:10F0300043FF019B1868401C1860196927872763E4
:10F040006162E663266467641D498C42029A07D1B7
:10F0500020681C49884220D11C48012101601868A1
:10F0600050B11348101A80101949414301208840BB
:10F0700018490A6802430A6003B0F0BD17A00E49A0
:10F08000C622FFF7F7F814480B49C922FFF7F2F838
:10F0900008480949CA22FFF7EDF80B48064940F233
:10F0A0000A12FFF7E7F8C046F8FD011088FB0110CF
:10F0B000E40B0210AB09021070090210E0FF0FFF11
:10F0C000881A01300000075051090210FC1A013063
:10F0D000B76DDBB6041B01300D06021028696E7493
:10F0E000296F626A2D3E73657269616C2E7561725B
:10F0F0007420213D204E430003688D4A1A409369D5
:10F100001B02FCD411603421405C800703D5506899
:10F110000221014351607047E0FF0FFFF0B581B05D
:10F120000446FEF72DFD2068C068804760683A21DC
:10F13000415CF9B93925012141554168A9B1204601
:10F1400000F0F8F86068026B436B4168C0C9083989
:10F15000921BBB4109D3CA68426003681BB188682F
:10F16000984760684268002AE9D10021415520464D
:10F17000FFF702FE01B0F0BC01BC8646FEF740BDC1
:10F1800080B500F001F880BDB0B50446FEF72CFF55
:10F19000FEF7F6FC204600F0CDF86068046B456B86
:10F1A000FEF72EFD20462946B0BD00009F480121F4
:10F1B000016000F0F5B9C0460A48406800F08CB81C
:10F1C00010B508484468606B1121084202D0E06C19
:10F1D0008047606B800700D410BDA06C10BC02BCDF
:10F1E0008E4600479CD200300A48406800F074B850
:10F1F00010B508484468606B1121084202D0E06CE9
:10F200008047606B800700D410BDA06C10BC02BCAE
:10F210008E460047B8D200300A48406800F05CB81B
:10F2200010B508484468606B1121084202D0E06CB8
:10F230008047606B800700D410BDA06C10BC02BC7E
:10F240008E460047D4D200300A48406800F044B8E7
:10F2500010B508484468606B1121084202D0E06C88
:10F260008047606B800700D410BDA06C10BC02BC4E
:10F270008E460047F0D200300A48406800F02CB8B3
:10F2800010B508484468606B1121084202D0E06C58
:10F290008047606B800700D410BDA06C10BC02BC1E
:10F2A0008E4600470CD300300A48406800F014B87E
:10F2B00010B508484468606B1121084202D0E06C28
:10F2C0008047606B800700D410BDA06C10BC02BCEE
:10F2D0008E46004728D30030B0B504460068144D70
:10F2E0000540E86941F2001108420CD0696811201C
:10F2F00081436960A26A32B13421615C014202D06B
:10F30000E06A00219047E86980050CD56868022111
:10F3100088436860A26A32B13420205C800702D53D
:10F32000E06A01219047E869E861A869A861B0BD79
:10F33000E0FF0FFFF0B585B0044646683A20305C28
:10F3400000286CD12068406880476168096A88425B
:10F3500065D0316A3062401AB168F468044073487D
:10F36000814201D1002354E00391704A00212046DC
:10F3700004910B46F9F7AEF80D463B21775C002F60
:10F380000290294618D03A46F9F793F804460191BD
:10F390003A46F9F77EF8029A101A8D41B16A0918B7
:10F3A000B162F06A6841F062039D4A1B0246049B09
:10F3B0009A4124D2019B2CE0039A049BF9F7A2F80E
:10F3C00004460F46039A049BF9F784F83B46029AD9
:10F3D000101A8D41B16A4118B162F06A6841049D0A
:10F3E000039FF062CA1B0246AA4112D3324628325A
:10F3F000C91B1160A8415060641C6B4109E0324692
:10F400002832491B116098415060641C0198584192
:10F410000346306B00193063706B5841706305B060
:10F42000F0BDC04601480121016070470810055039
:10F430003A4804210160BFF34F8FBFF36F8F7047CD
:10F440000248042101606E480160704704E200E058
:10F4500080B5324804210160BFF34F8FBFF36F8F37
:10F460002F4800F025F958480021018080BDC04692
:10F4700000487047D40C0210B0B52748018839B154
:10F48000264804210160BFF34F8FBFF36F8FB0BDDB
:10F49000012505806904224C0022204600F01AF95B
:10F4A000204600F01DF91F4800F00EF91E4C2046C2
:10F4B000FCF794FA1D4AB0FBF2F3591E802920D2C2
:10F4C0005A43801A22D10320C006014321604B48D1
:10F4D000606031480068C821304A42500F4804211A
:10F4E0000160BFF34F8FBFF36F8F6807216801433F
:10F4F0002160A80721680143216020688001FCD5B4
:10F50000B0BD0BA019496B22FEF7B4FE18A0174935
:10F510006C22FEF7AFFEC046001B013084E100E024
:10F520000400005F040000040010055040420F007A
:10F53000287072657363616C655F74696D657220B4
:10F54000213D202875696E7433325F7429202D3176
:10F5500029202626207072657363616C655F74696B
:10F560006D6572203C3D203132370000D609021013
:10F5700028636C6B5F74696D65722025204E555F42
:10F58000544D52434C4B5F5045525F5345432920E5
:10F590003D3D20300000000008ED00E0ADF101101D
:10F5A0000248016809B102480847704798D2003004
:10F5B000A80C021080B50448008808B9FFF75CFF6A
:10F5C0000248006880BDC046001B01300C10055089
:10F5D000084901224A60084B04221A60022800D818
:10F5E0000220064B984200D3184608600448026087
:10F5F0007047C0460410055084E200E0FFFFFF00A2
:10F6000004E100E070B50446FEF74CFB0546FFF749
:10F61000B7FD06462846FFF7B3FD801BA042F9D38D
:10F6200070BDB0B514460D46FDF73AFC38B101681F
:10F63000CB68294622469847002802DBB0BD092442
:10F6400000E04442F8F7CAFE04600020C043B0BDA9
:10F6500003B40148019001BDB170010003B4014839
:10F66000019001BD7970010003B40148019001BD12
:10F670008170010003B40148019001BD7170010067
:10F6800003B40148019001BD9970010003B4014821
:10F69000019001BDA170010003B40148019001BDBA
:10F6A000A970010003B40148019001BD91700100EF
:10F6B00003B40148019001BDC170010003B40148C9
:10F6C000019001BDF970010003B40148019001BD32
:10F6D000F170010003B40148019001BDE170010027
:10F6E00003B40148019001BDC970010003B4014891
:10F6F000019001BDE970010003B40148019001BD12
:10F700006170010003B40148019001BD4170010026
:10F7100003B40148019001BD3170010003B40148F8
:10F72000019001BD5170010003B40148019001BD79
:10F730003970010003B40148019001BD5970010006
:10F7400003B40148019001BD4970010003B40148B0
:10F75000019001BD2970010003B40148019001BD71
:10F760006970010003B40148019001BD11710100ED
:10F77000F0B4040C8BB2264682B25E431046584366
:10F780000D0C370C360400218019164679416E4362
:10F79000370C36048019264679416E438919F0BC2E
:10F7A000704700004900CA020243100000D0042044
:10F7B0004A0D01D001221043044A490D914201D162
:10F7C00002210843012800D105207047FF070000EF
:10F7D00030380A2801D2012070470020704710B548
:10F7E0008A68002A02DCF9F709FD10BD521E8A6002
:10F7F0004A68C0B2531C4B60107010BD10B5002990
:10F800000AD00878002807D005487844F9F7AAFA02
:10F81000002801D0002010BD0248784410BD00002F
:10F82000F2140000EA14000010B500290AD008788C
:10F83000002807D005487844F9F794FA002801D049
:10F84000002010BD0248784410BD0000D61500000D
:10F85000CE15000003B402487844844603BC6047D8
:10F860002DA2FFFF03B402487844844603BC6047DE
:10F8700095A4FFFF303132333435363738394142C1
:10F880004344454640305800303132333435363702
:10F8900038396162636465664030780004000008AE
:10F8A0000000000000000002000100001000000045
:10F8B00000000000000000003031323334353637AC
:10F8C0003839616263646566787000303132333490
:10F8D00035363738394142434445465850000000D8
:10F8E00002400000000000A00000000005400000F1
:10F8F000000000C8000000000C4000000000409C18
:10F9000000000000194000000020BCBE0000000004
:10F9100034400000BFC91B8E00000004B540000049
:10F92000504BCFD06607E2CF010000006C410000D1
:10F930003E8251AADFEEA73401000000D942000048
:10F94000DCB5A0E23A301F97FFFFFFFFB44500008F
:10F95000FD25A0C8E9A3C14FFFFFFFFFFF3F000047
:10F960000000008000000000FF3F00000000008059
:10F97000000000002000000020000000100A02101B
:10F980000040000000000000B0D90030004000003E
:10F9900000000000B0D90030982F8A42914437719E
:10F9A000CFFBC0B5A5DBB5E95BC25639F111F15902
:10F9B000A4823F92D55E1CAB98AA07D8015B831244
:10F9C000BE853124C37D0C55745DBE72FEB1DE80F0
:10F9D000A706DC9B74F19BC1C1699BE48647BEEF1F
:10F9E000C69DC10FCCA10C246F2CE92DAA84744AAA
:10F9F000DCA9B05CDA88F97652513E986DC631A820
:10FA0000C82703B0C77F59BFF30BE0C64791A7D5FE
:10FA10005163CA0667292914850AB72738211B2E86
:10FA2000FC6D2C4D130D385354730A65BB0A6A766E
:10FA30002EC9C281852C7292A1E8BFA24B661AA87A
:10FA4000708B4BC2A3516CC719E892D1240699D68A
:10FA500085350EF470A06A1016C1A419086C371E03
:10FA60004C774827B5BCB034B30C1C394AAAD84EE1
:10FA70004FCA9C5BF36F2E68EE828F746F63A5781C
:10FA80001478C8840802C78CFAFFBE90EB6C50A4AF
:10FA9000F7A3F9BEF27871C60C01000000D0005047
:10FAA00000000900FFFFFFFFFFFFFFFF0000000055
:10FAB0000101000000D000503000000006040000EA
:10FAC00000D0005000000003FFFFFFFFFFFFFFFF1B
:10FAD000000000000001000000D000500300000002
:10FAE0000704000000D0005000000030FFFFFFFFBF
:10FAF000FFFFFFFF000000000201000000D00050E7
:10FB0000000300000204000000D0005000030000C9
:10FB1000FFFFFFFFFFFFFFFF0000000003010000E9
:10FB200000D00050003000000304000000D000505E
:10FB300000300000FFFFFFFFFFFFFFFF000000009D
:10FB40000401000000D00050000003000404000085
:10FB500000D0005000000300FFFFFFFFFFFFFFFF8A
:10FB6000000000000501000000D00050000030003F
:10FB70000504000000D0005000003000FFFFFFFF30
:10FB8000FFFFFFFF00000000000000000000075022
:10FB900007000000020000000010175000080000DD
:10FBA00002100100001017500008000002000000C1
:10FBB000004047500007000002400100004047504D
:10FBC00000070000040000000000075000000B00C8
:10FBD000040000000050575000000800060000001C
:10FBE0000000075000000007080000000010175038
:10FBF000070000000D0000000040475000003000EA
:10FC00000F0000000000075000000030000100005D
:10FC100000202750070000000201000000101750CC
:10FC200000060000040100000020275000000C0026
:10FC300004010000005057500000070006010000BA
:10FC400000101750000000060801000000000750D7
:10FC5000050000000A0100000040475000060000B7
:10FC60000C01000000000750000006000E0100001B
:10FC7000003037500000000700020000002027502D
:10FC8000080000000202000000303750000B0000A6
:10FC90000402000000202750000008000422010098
:10FCA00000202750000008000402000000404750D8
:10FCB00000000B00044201000040475000000B0010
:10FCC0000602000000404750000000050802000046
:10FCD00000101750080000000902000000303750E3
:10FCE000700000000B020000000007500030000010
:10FCF0000003000000303750050000000203000040
:10FD00000000075000090000060300000010175013
:10FD1000000000030A030000001017500003000059
:10FD20000C03000000202750000007000004000022
:10FD30000030375007000000060400000050575004
:10FD40000000000809040000002027507000000097
:10FD50000B04000000303750007000000F0400005A
:10FD6000002027500000003001050000000007506F
:10FD700040000000010500000010175020000000A6
:10FD80000205000000000750000300000505000008
:10FD900000202750000020000605000000404750CA
:10FDA000000000060A050000005057500006000041
:10FDB0000907000000101750A00000000B0700000A
:10FDC00000000750008000000B07010000000750F2
:10FDD000008000000B07000000404750007000004A
:10FDE0000B4701000040475000700000FFFFFFFF7D
:10FDF000FFFFFFFF000000000100000000000750AF
:10FE00007000000003000000001017500080000088
:10FE100003100100001017500080000003000000D4
:10FE20000040475000700000034001000040475070
:10FE30000070000005000000000007500000B00046
:10FE4000050000000050575000008000070000002F
:10FE5000000007500000007009000000001017505B
:10FE6000700000000C00000000404750000003003C
:10FE70000E00000000000750000000030101000018
:10FE800000202750700000000301000000101750F0
:10FE90000060000005010000002027500000C000A5
:10FEA00005010000005057500000700007010000DD
:10FEB000001017500000006009010000000007500A
:10FEC000500000000B01000000404750006000009F
:10FED0000D01000000000750000060000F0100004D
:10FEE0000030375000000070010200000020275051
:10FEF00080000000030200000030375000B0000016
:10FF000005020000002027500000800005220100AB
:10FF100000202750000080000502000000404750EC
:10FF20000000B00005420100004047500000B00052
:10FF30000702000000404750000000500A02000085
:10FF400000303750000700000C020000000007508E
:10FF5000000003000D020000002027500000700088
:10FF60000103000000303750500000000303000080
:10FF70000000075000900000070300000010175019
:10FF8000000000300B03000000101750003000008C
:10FF9000010400000030375070000000070400002A
:10FFA0000050575000000080080400000020275037
:10FFB000070000000A04000000303750000700006E
:10FFC0000D04000000101750000080000E04000017
:10FFD000002027500000000300050000000007502B
:10FFE000040000000005000000101750020000008F
:10FFF0000305000000000750003000000405000069
:020000041002E8
:100000000020275000000200070500000040475074
:10001000000000600B050000005057500060000019
:1000200008070000001017500A0000000A0700002F
:1000300000000750000800000A07010000000750F8
:10004000000800000A0700000040475000070000B9
:100050000A4701000040475000070000FFFFFFFF74
:10006000FFFFFFFF00000000000000000000000094
:100070000000000000000000000000000000000080
:100080000000000000000000000000000000000070
:100090000000000000000000000000000000000060
:1000A00000000000000000000000000000D0005030
:1000B00006FF4307000020000000000106000000CA
:1000C0004000000000000000FFFFFFFF00000000F4
:1000D0000000000000000000000000000000000020
:1000E00000000000C5C60110CDC60110D5C6011024
:1000F000DDC60110E5C60110EDC60110F5C6011000
:10010000FDC6011000000000B71DC1046E3B82094E
:10011000D926430DDC7604136B6BC517B24D861AD6
:100120000550471EB8ED08260FF0C922D6D68A2FF3
:1001300061CB4B2B649B0C35D386CD310AA08E3C12
:10014000BDBD4F3870DB114CC7C6D0481EE093458B
:10015000A9FD5241ACAD155F1BB0D45BC29697565A
:10016000758B5652C836196A7F2BD86EA60D9B63C5
:1001700011105A6714401D79A35DDC7D7A7B9F7056
:10018000CD665E74E0B6239857ABE29C8E8DA1914C
:10019000399060953CC0278B8BDDE68F52FBA582A2
:1001A000E5E66486585B2BBEEF46EABA3660A9B72F
:1001B000817D68B3842D2FAD3330EEA9EA16ADA44E
:1001C0005D0B6CA0906D32D42770F3D0FE56B0DD7D
:1001D000494B71D94C1B36C7FB06F7C32220B4CE5E
:1001E000953D75CA28803AF29F9DFBF646BBB8FB49
:1001F000F1A679FFF4F63EE143EBFFE59ACDBCE8CA
:100200002DD07DEC77708634C06D4730194B043D9E
:10021000AE56C539AB0682271C1B4323C53D002EB5
:100220007220C12ACF9D8E1278804F16A1A60C1B7A
:1002300016BBCD1F13EB8A01A4F64B057DD0080831
:10024000CACDC90C07AB9778B0B6567C69901571CA
:10025000DE8DD475DBDD936B6CC0526FB5E6116239
:1002600002FBD066BF469F5E085B5E5AD17D1D577C
:100270006660DC5363309B4DD42D5A490D0B1944F5
:10028000BA16D84097C6A5AC20DB64A8F9FD27A50F
:100290004EE0E6A14BB0A1BFFCAD60BB258B23B601
:1002A0009296E2B22F2BAD8A98366C8E41102F8336
:1002B000F60DEE87F35DA9994440689D9D662B90ED
:1002C0002A7BEA94E71DB4E0500075E4892636E9FC
:1002D0003E3BF7ED3B6BB0F38C7671F7555032FA3D
:1002E000E24DF3FE5FF0BCC6E8ED7DC231CB3ECF00
:1002F00086D6FFCB8386B8D5349B79D1EDBD3ADC69
:100300005AA0FBD8EEE00C6959FDCD6D80DB8E6004
:1003100037C64F643296087A858BC97E5CAD8A7386
:10032000EBB04B77560D044FE110C54B383686467F
:100330008F2B47428A7B005C3D66C158E440825562
:10034000535D43519E3B1D252926DC21F0009F2C47
:10035000471D5E28424D1936F550D8322C769B3F0A
:100360009B6B5A3B26D6150391CBD40748ED970AD1
:10037000FFF0560EFAA011104DBDD014949B9319A6
:100380002386521D0E562FF1B94BEEF5606DADF878
:10039000D7706CFCD2202BE2653DEAE6BC1BA9EBD2
:1003A0000B0668EFB6BB27D701A6E6D3D880A5DE3B
:1003B0006F9D64DA6ACD23C4DDD0E2C004F6A1CD1E
:1003C000B3EB60C97E8D3EBDC990FFB910B6BCB419
:1003D000A7AB7DB0A2FB3AAE15E6FBAACCC0B8A78E
:1003E0007BDD79A3C660369B717DF79FA85BB492D5
:1003F0001F4675961A163288AD0BF38C742DB0819A
:10040000C330718599908A5D2E8D4B59F7AB085496
:1004100040B6C95045E68E4EF2FB4F4A2BDD0C47E5
:100420009CC0CD43217D827B9660437F4F46007206
:10043000F85BC176FD0B86684A16476C9330046101
:10044000242DC565E94B9B115E565A158770191806
:10045000306DD81C353D9F0282205E065B061D0B69
:10046000EC1BDC0F51A69337E6BB52333F9D113E88
:100470008880D03A8DD097243ACD5620E3EB152DC5
:1004800054F6D4297926A9C5CE3B68C1171D2BCCBB
:10049000A000EAC8A550ADD6124D6CD2CB6B2FDFB1
:1004A0007C76EEDBC1CBA1E376D660E7AFF023EA42
:1004B00018EDE2EE1DBDA5F0AAA064F4738627F93D
:1004C000C49BE6FD09FDB889BEE0798D67C63A8018
:1004D000D0DBFB84D58BBC9A62967D9EBBB03E93ED
:1004E0000CADFF97B110B0AF060D71ABDF2B32A68C
:1004F0006836F3A26D66B4BCDA7B75B8035D36B5B9
:10050000B440F7B10000000000000000B9CD0110B8
:10051000A9CD0110D1C701100DCA011099CE01104B
:1005200015C901103DCA0110FDC901109DCE011071
:1005300045D201105DD201104DD2011055D20110EB
:1005400063D3011065D2011091D2011069D301105B
:10055000FFD201107DD20110F9C901100000000086
:100560000000000051CE011003CE0110E5CD0110B6
:10057000FBCD0110EDCD0110F7CD011025CE0110FE
:10058000FFCD011029CE011041CE0110F1CD011097
:100590004BCE011039CE011033CE01101FCE011009
:1005A0000DCE011089D2011007CE011019CE011015
:1005B0008DD201103FCE01100000000000000000AD
:1005C000C9CF0110C5CF01106DCF01102F73746416
:1005D000657272002F737464696E002F7374646F98
:1005E00075740000001BB7000000000000800000D0
:1005F000001BB70000000000000000000000000029
:1006000000000000E38C01105F7364685F6D6F642D
:10061000696E697420213D204E554C4C002E5C645F
:100620007269766572735C73746F726167655C433F
:100630004F4D504F4E454E545F4E5553445C4E7592
:100640005344426C6F636B4465766963652E6370D7
:10065000700063726320213D204E554C4C002E2FBC
:100660006D6265642D6F732F647269766572735C59
:100670004D6265644352432E68006F626A2D3E707E
:10068000696E20213D202850696E4E616D65294EAE
:1006900043002E2F6D6265642D6F732F7461726736
:1006A0006574732F5441524745545F4E55564F540D
:1006B0004F4E2F5441524745545F4D323335342FFE
:1006C0006770696F5F6F626A6563742E680052615C
:1006D0006E206F7574206F6620435468756E6B20B2
:1006E000656E74726965732E20496E6372656173FD
:1006F00065204D4245445F434F4E465F504C415448
:10070000464F524D5F435448554E4B5F434F554EF5
:10071000545F4D415820746F206669782074686971
:1007200073206572726F72000A2D2D204D62656410
:100730004F53204572726F7220496E666F202D2DC7
:100740000A004B65726E656C204572726F723A20BA
:10075000307825582C20000A0A2B2B204D62656426
:100760004F53204572726F7220496E666F202B2B9B
:100770000A4572726F72205374617475733A203037
:1007800078255820436F64653A202564204D6F64B6
:10079000756C653A2025640A4572726F72204D654A
:1007A00073736167653A20000A466F72206D6F723D
:1007B0006520696E666F2C2076697369743A2068CB
:1007C000747470733A2F2F6D6265642E636F6D2F92
:1007D000732F6572726F723F6572726F723D3078FF
:1007E00025303858267467743D4E555F4D32333589
:1007F000345F4E5053415F4E53000A4572726F7220
:100800002056616C75653A2030782558000A4C6F87
:10081000636174696F6E3A203078255800286775D7
:100820006172642026204358415F47554152445F1E
:100830004D41534B29203D3D204358415F47554191
:1008400052445F494E49545F494E5F50524F4752A0
:10085000455353002E5C6D6265642D6F735C706C44
:100860006174666F726D5C736F757263655C6D62E7
:1008700065645F72657461726765742E6370700081
:1008800028706172697479203D3D205061726974ED
:10089000794E6F6E6529207C7C20287061726974A6
:1008A00079203D3D205061726974794F646429203C
:1008B0007C7C2028706172697479203D3D205061F4
:1008C000726974794576656E29207C7C2028706178
:1008D00072697479203D3D20506172697479466F68
:1008E000726365643129207C7C2028706172697490
:1008F00079203D3D20506172697479466F7263655D
:100900006430290028646174615F62697473203DFA
:100910003D203529207C7C2028646174615F6269F8
:100920007473203D3D203629207C7C20286461742E
:10093000615F62697473203D3D203729207C7C20F3
:1009400028646174615F62697473203D3D203829B9
:10095000006F626A2D3E73657269616C2E756172FB
:1009600074203D3D20535444494F5F55415254003B
:100970002E5C6D6265642D6F735C74617267657463
:10098000735C5441524745545F4E55564F544F4E39
:100990005C5441524745545F4D323335345C736586
:1009A0007269616C5F6170692E63006D6F64696E5E
:1009B00069742D3E6D6F646E616D65203D3D20282C
:1009C000696E7429206F626A2D3E73657269616C6D
:1009D0002E75617274002E5C6D6265642D6F735CA0
:1009E000746172676574735C5441524745545F4E3D
:1009F00055564F544F4E5C5441524745545F4D320B
:100A00003335345C75735F7469636B65722E630094
:100A100053746F72616765456E63323536484D4178
:100A2000435348413235365349474E415455524558
:100A3000005B455252205D204153534552540D0AEC
:100A4000005B444247205D204669726D77617265A4
:100A50002073697A6520726F756E646564207570A5
:100A600020746F20746865206E65617265737420F0
:100A7000736563746F7220626F756E646172792042
:100A80006973206C6172676572207468616E20748E
:100A90006865206D6178696D756D206170706C6935
:100AA000636174696F6E2073697A650D0A0046612F
:100AB000696C656420746F206A756D7020746F2096
:100AC0006170706C69636174696F6E210D0A005BFF
:100AD000444247205D204669726D776172652075DA
:100AE0007064617465206661696C65640D0A005507
:100AF000706461746520696D61676520696E7465F5
:100B0000677269747920636865636B206661696CDC
:100B100065640D0A005B444247205D204E657720E6
:100B2000616374697665206669726D7761726520AC
:100B300069732076616C69640D0A005B455252202E
:100B40005D20416374697665206669726D776172B4
:100B50006520696E76616C69640D0A004E6F2055E0
:100B6000706461746520696D6167650D0A00557078
:100B70006461746520696D61676520746F6F206CB6
:100B8000617267650D0A005B444247205D20557025
:100B90006461746520616374697665206669726D4D
:100BA000776172650D0A005B444247205D20416316
:100BB00074697665206669726D77617265207570FB
:100BC0002D746F2D646174650D0A00557064617435
:100BD0006520696D616765206973206F6C6465725B
:100BE0000D0A000000000750103D006F00000300D8
:100BF0000000000010000004240000009CD200301F
:100C000000101750913D406F0000300000000000C0
:100C10001100000425000000B8D200300020275049
:100C2000123C8C6F00000003000000001200000462
:100C300030000000D4D2003000303750933CCC6FED
:100C4000000000300000000013000004310000002C
:100C5000F0D2003000404750143D8C7F000000036C
:100C600000000000140000044A0000000CD3003013
:100C700000505750953DCC7F000000300000000030
:100C8000150000044B00000028D30030FFFFFFFFD9
:100C90000000000000000000000000000000000054
:100CA0000000000000000000B00C0210C01901306C
:100CB0007DE90110B5F5011031F4011025F40110A2
:100CC000D1F5011041F4011071E9011071F4011026
:100CD0000000000040420F00180000002C0E02101F
:100CE00010D20030340100000CA80110980E021040
:100CF00044D30030C44700005482011010010000AA
:100D000043000000F8FFFFFF0040404040404040EB
:100D100040404141414141404040404040404040CE
:100D20004040404040404040400502020202020272
:100D300002020202020202020220202020202020C1
:100D400020202002020202020202909090909090D5
:100D50001010101010101010101010101010101093
:100D60001010101002020202020288888888888807
:100D700008080808080808080808080808080808F3
:100D800008080808020202024000000000000000FB
:100D90000000000000000000000000000000000053
:100DA0000000000000000000000000000000000043
:100DB0000000000000000000000000000000000033
:100DC0000000000000000000000000000000000023
:100DD0000000000000000000000000000000000013
:100DE0000000000000000000000000000000000003
:100DF00000000000000000000000000000000000F3
:100E00000000000000000000000000001C000000C6
:100E100043000000F8FFFFFF0C0000000E00000080
:100E20000F0000002E00000001AFFFFFC105149D60
:100E3000A801104B7DA9181AF1085AE52442302C5C
:100E40006CDC02049AFF0101348F640502101DF16D
:100E50007C290929041AB9141AC104A30405691CC0
:100E60001AE9181AF1040B1006071C1E19F20110DA
:100E700021040B1008091C1A49181A51040B100AF6
:100E80000B1C1A79181A81040B100C0D1C1AA918C6
:080E90001AB104230E0F00004B
:040000051001821153
:00000001FF
